:1000000012C4000041C400003FC400003DC4000011
:100010003BC4000039C4000037C4000035C40000F0
:1000200033C4000031C400002FC400002DC4000000
:100030000C946B1F29C4000027C4000025C40000D5
:1000400023C4000021C400001FC400001DC4000020
:100050001BC4000019C4000017C400000C94E7235F
:1000600013C400000C94A31B0C947A1B0DC4000055
:100070000BC4000009C4000007C4000005C4000050
:1000800003C4000001C40000FFC30000FDC3000062
:10009000FBC30000F9C30000F7C300000C94D91B98
:1000A000F3C30000F1C30000EFC30000EDC3000084
:1000B000EBC30000E9C30000E7C30000E5C3000094
:1000C000E3C30000E1C30000DFC30000DDC30000A4
:1000D000DBC30000D9C30000D7C30000D5C30000B4
:1000E000D3C300006C116F115E1162116811A6116B
:1000F000731177117D11811185118B118F1193115E
:10010000A61199119D11A11100407A10F35A00A077
:10011000724E18090010A5D4E80000E876481700D0
:1001200000E40B54020000CA9A3B000000E1F50510
:10013000000080969800000040420F000000A0865A
:1001400001000000102700000000E803000000008C
:100150006400000000000A00000000000100000030
:1001600000002C76D888DC674F0823DFC1DFAE594A
:10017000E1B1B796E5E3E453C63AE651997696E8DD
:10018000E6C28426EB898C9B62ED407C6FFCEFBC61
:100190009C9F40F2BAA56FA5F490055A2AF75C938C
:1001A0006B6CF9676DC11BFCE0E40D47FEF520E6C2
:1001B000B500D0ED902E0300943577050080841EA5
:1001C000080000204E0A000000C80C333333330F00
:1001D000986E12831141EF8D2114893BE65516CF9D
:1001E000FEE6DB18D1844B381BF77C1D901DA4BBA9
:1001F000E424203284725E228100C9F124ECA1E55E
:100200003D2700002100240027002A002D00300097
:10021000330001010000040107010A010000200071
:100220002300260029002C002F00320000010000CE
:1002300003010601090100000A0B02090C0D0E085A
:10024000070304010000000000000000000000009F
:10025000000000000000000000000000000000009E
:10026000000012111000000000000000000000005B
:10027000000000000000000000000000000000007E
:10028000003E5B4F5B3E3E6B4F6B3E1C3E7C3E1C1C
:10029000183C7E3C181C577D571C1C5E7F5E1C0062
:1002A000183C1800FFE7C3E7FF0018241800FFE719
:1002B000DBE7FF30483A060E2629792926407F05DC
:1002C0000507407F05253F5A3CE73C5A7F3E1C1CF2
:1002D00008081C1C3E7F14227F22145F5F005F5FB2
:1002E00006097F017F006689956A6060606060949E
:1002F000A2FFA29408047E040810207E20100808A3
:100300002A1C08081C2A08081E101010100C1E0CAD
:100310001E0C30383E3830060E3E0E06000000003F
:100320000000005F00000007000700147F147F1426
:10033000242A7F2A1223130864623649562050006B
:1003400008070300001C2241000041221C002A1C57
:100350007F1C2A08083E0808008070300008080842
:100360000808000060600020100804023E51494562
:100370003E00427F400072494949462141494D3380
:100380001814127F1027454545393C4A49493141E7
:10039000211109073649494936464949291E0000B5
:1003A000140000004034000000081422411414140A
:1003B0001414004122140802015909063E415D59F6
:1003C0004E7C1211127C7F494949363E41414122FF
:1003D0007F4141413E7F494949417F090909013E29
:1003E000414151737F0808087F00417F4100204050
:1003F000413F017F081422417F404040407F021C62
:10040000027F7F0408107F3E4141413E7F09090978
:10041000063E4151215E7F09192946264949493244
:1004200003017F01033F4040403F1F2040201F3F0A
:100430004038403F6314081463030478040361598F
:10044000494D43007F4141410204081020004141D1
:10045000417F04020102044040404040000307087D
:100460000020545478407F28444438384444442879
:10047000384444287F385454541800087E09021820
:10048000A4A49C787F0804047800447D40002040A8
:10049000403D007F1028440000417F40007C0478EC
:1004A00004787C080404783844444438FC18242434
:1004B0001818242418FC7C080404084854545424B4
:1004C00004043F44243C4040207C1C2040201C3C31
:1004D0004030403C44281028444C9090907C446428
:1004E000544C4400083641000000770000004136BB
:1004F000080002010204023C2623263C1EA1A16141
:10050000123A4040207A3854545559215555794172
:100510002254547842215554784020545579400C47
:100520001E5272123955555559395454545939552A
:100530005454580000457C410002457D420001456D
:100540007C407D1211127DF0282528F07C54554501
:10055000002054547C547C0A097F4932494949326D
:100560003A4444443A324A4848303A4141217A3A7E
:1005700042402078009DA0A07D3D4242423D3D404A
:1005800040403D3C24FF2424487E4943662B2FFCF9
:100590002F2BFF0929F620C0887E090320545479A7
:1005A000410000447D413048484A32384040227A78
:1005B000007A0A0A727D0D19317D2629292F2826F5
:1005C0002929292630484D402038080808080808FD
:1005D0000808382F10C8ACBA2F102834FA00007B56
:1005E000000008142A142222142A14085500550069
:1005F00055AA55AA55AAFF55FF55FF000000FF0058
:10060000101010FF00141414FF001010FF00FF1052
:1006100010F010F0141414FC001414F700FF000084
:10062000FF00FF1414F404FC141417101F10101F03
:10063000101F1414141F00101010F0000000001FF1
:10064000101010101F10101010F010000000FF10FC
:100650001010101010101010FF10000000FF1400F8
:1006600000FF00FF00001F10170000FC04F414142A
:100670001710171414F404F40000FF00F7141414F6
:1006800014141414F700F7141414171410101F1076
:100690001F141414F4141010F010F000001F101F99
:1006A0000000001F14000000FC140000F010F01007
:1006B00010FF10FF141414FF141010101F0000007E
:1006C00000F010FFFFFFFFFFF0F0F0F0F0FFFFFF82
:1006D0000000000000FFFF0F0F0F0F0F38444438D9
:1006E00044FC4A4A4A347E02020606027E027E0228
:1006F00063554941633844443C04407E201E200633
:10070000027E020299A5E7A5991C2A492A1C4C726F
:1007100001724C304A4D4D303048784830BC625AF6
:10072000463D3E494949007E0101017E2A2A2A2A86
:100730002A44445F444440514A444040444A514062
:100740000000FF0103E080FF000008086B6B083623
:1007500012362436060F090F060000181800000094
:100760001010003040FF0101001F01011E00191D83
:100770001712003C3C3C3C0000000000010210202D
:1007800020080810204010204080020102010804C7
:10079000020101020408102040808040201008045B
:1007A00002018004020180402010080402010804B4
:1007B00002010102040810204080010204081020F8
:1007C000408000002200250028002B002E00310070
:1007D000340002010000050108010B0105050505B3
:1007E000070508080808020202020A0A08080404A9
:1007F00004040101010101010101030303030303D7
:100800000303040707070C0C0C0C0C0C0C0C020265
:10081000020206060606060606060B0B0B0B0B0B62
:100820000B0B7A2B722B11241FBECFEFD1E2DEBF50
:10083000CDBF00E00CBF15E0A0E0B2E0EAEFF8E6C3
:1008400000E00BBF02C007900D92A03EB107D9F7A0
:1008500027E0A0EEB5E001C01D92A03CB207E1F791
:1008600014E0C2E1D4E000E006C021970109802F26
:10087000FE010E940A32C131D10780E00807A9F7C2
:100880000E9431240C946C34BBCB0895FC0163703E
:10089000658B8481958126813781613039F06330A1
:1008A00029F09187808733872287089531872087B1
:1008B0009387828708956F927F928F929F92AF92D3
:1008C000BF92CF92DF92EF92FF920F931F93CF933D
:1008D000DF93EC014B015A0169013801E881F9818C
:1008E0000284F385E02D1995E881F9810288F38966
:1008F000E02D87019601A501B401CE011995A5014E
:10090000460D571D41505109E881F9810288F3894C
:10091000E02D9601B401CE011995E881F981008896
:10092000F189E02D9301A501B401CE011995C80C00
:10093000D91CB60161507109E881F9810088F189FB
:10094000E02D9301A501CE011995E881F981068872
:10095000F789E02DCE01DF91CF911F910F91FF908C
:10096000EF90DF90CF90BF90AF909F908F907F904F
:100970006F9019948F929F92AF92BF92CF92DF9215
:10098000EF92FF920F931F93CF93DF934C016B0174
:100990005A01E901DC01ED91FC916217730781F4C2
:1009A0000417150724F48B2D5801042F182F0A194A
:1009B0001B0998012F5F3F4F048CF58DE02D12C06D
:1009C0004017510709F52617370724F48D2D6901C3
:1009D000C62FD82F9E012C193D092F5F3F4F068C43
:1009E000F78DE02D8701A501B601C4011995DF91AE
:1009F000CF911F910F91FF90EF90DF90CF90BF901C
:100A0000AF909F908F9008950284F385E02D199503
:100A1000D401ED91FC910488F589E02D9E01A5019A
:100A2000B601C4011995D401ED91FC910688F789AE
:100A3000E02DC401DF91CF911F910F91FF90EF90B6
:100A4000DF90CF90BF90AF909F908F901994EF92CE
:100A5000FF920F931F93DC011A960D911C911B9727
:100A600018962D913C911997ED91FC9100A0F1A160
:100A7000E02D7B0140E050E060E070E019951F91AF
:100A80000F91FF90EF9008954F925F926F927F9237
:100A90008F929F92AF92BF92CF92DF92EF92FF928E
:100AA0000F931F93CF93DF936C012B015A013901F0
:100AB0004801DC01ED91FC910284F385E02D19954C
:100AC000E201640C751CD601ED91FC91C615D705A9
:100AD0005CF40088F189E02D87019401A501BE0135
:100AE000C60119952196EFCF0688F789E02DC6013A
:100AF000DF91CF911F910F91FF90EF90DF90CF90FA
:100B0000BF90AF909F908F907F906F905F904F902D
:100B100019948F929F92AF92BF92CF92DF92EF92F1
:100B2000FF920F931F93CF93DF93EC015B014A0178
:100B30006901E881F9810284F385E02D1995950119
:100B40002C0D3D1D21503109E881F9810488F5897A
:100B5000E02D78018401A401B501CE011995E88149
:100B6000F9810688F789E02DCE01DF91CF911F91A1
:100B70000F91FF90EF90DF90CF90BF90AF909F903C
:100B80008F9019948F929F92AF92BF92CF92DF92E3
:100B9000EF92FF920F931F93CF93DF93EC015B01D2
:100BA0004A0169017801E881F9810284F385E02D29
:100BB0001995C80CD91C860101501109E881F981E9
:100BC0000488F589E02D9501A401B501CE011995A0
:100BD000E881F9810688F789E02DCE01DF91CF9178
:100BE0001F910F91FF90EF90DF90CF90BF90AF904B
:100BF0009F908F901994EF92FF920F931F93DC01B7
:100C0000ED91FC9100A0F1A1E02D19951F910F919C
:100C1000FF90EF9008950F931F93DC01ED91FC91ED
:100C2000068CF78DE02D19951F910F910895AF92C5
:100C3000BF92CF92EF92FF920F931F93CF93DF93C8
:100C4000EC01262F888D998D009709F040C06A30FD
:100C500059F41D861C862C898E859F8538E0239F3C
:100C6000800D911D112441C06D3009F4AAC08E89F8
:100C70008823C1F03C898C859D8546E0349F800D9A
:100C8000911D112448855985481759075CF41D8624
:100C90001C868E859F8548E0349F800D911D112410
:100CA0009F878E87EA88FB88088919894E855F852A
:100CB0006C857D85CC88CE010E9468142C898C853A
:100CC0009D8536E0239F800D911D112442C06A301E
:100CD00079F41D861C862C89FC013696E4918E855C
:100CE0009F852E9F800D911D11249F878E8769C03F
:100CF0006D3009F466C0FC0134963491631708F432
:100D000060C03196E491E61708F45BC0FC013296AE
:100D100065917491422F50E0431B510937E0349F95
:100D20005001359FB00C1124A60EB71EF501329666
:100D300034913196E491332311F0E1110DC0F501A6
:100D40003496E4912C898C859D85E29F800D911DC0
:100D500011249D878C8735C0F501359644915E89B5
:100D6000552311F16C89E32FF0E0E40FF11D47FDED
:100D7000FA956E9FD0016F9FB00D11244C855D8553
:100D80004A0F5B1FE885F985E417F5076CF41D86AB
:100D90001C86FC013696E4918E859F856E9F800DA2
:100DA000911D11249F878E87EA88FB8808891989FD
:100DB0004E855F856C857D85CC88CE010E94681448
:100DC000BECF81E090E0DF91CF911F910F91FF9016
:100DD000EF90CF90BF90AF900895FC01A38DB48D9C
:100DE0009C9187A189238C93808591859C012150BA
:100DF00031098150A58DB68D2C9190A592239C939D
:100E000094E092B9A78DB0A12C9191A592239C93C7
:100E1000A78DB0A12C9195A1922B9C93A58DB68DF9
:100E20002C9194A1922B9C9332B9A78DB0A12C91B7
:100E300091A592239C93A78DB0A12C9195A1922B63
:100E40009C93A58DB68D2C9190A592239C9395E0B3
:100E500092B9A78DB0A12C9191A592239C93A78DB7
:100E6000B0A12C9195A1922B9C93A58DB68D2C9120
:100E700094A1922B9C9382B9A78DB0A19C9181A53E
:100E800089238C93A78DB0A19C9185A1892B8C93EC
:100E9000828593859C01215031098150A58DB68DA5
:100EA0002C9190A592239C9398E092B9A78DB0A124
:100EB0002C9191A592239C93A78DB0A12C9195A1E3
:100EC000922B9C93A58DB68D2C9194A1922B9C93E3
:100ED00032B9A78DB0A12C9191A592239C93A78D97
:100EE000B0A12C9195A1922B9C93A58DB68D2C91A0
:100EF00090A592239C9399E092B9A78DB0A12C91D3
:100F000091A592239C93A78DB0A12C9195A1922B92
:100F10009C93A58DB68D2C9194A1922B9C9382B914
:100F2000A78DB0A19C9181A589238C93A78DB0A199
:100F30009C9185A1892B8C93A38DB48D9C9183A1C9
:100F4000892B8C930895EF92FF920F931F93CF9369
:100F5000DF93EC01CB017A01EB8DFC8D50814FA129
:100F6000452340834A8D4111B6C14D89423089F0F5
:100F7000433021F1413091F54FEE50E0DA01A01BF2
:100F8000B10B4E195F09FA0189019A017B01CD016C
:100F900027C06FEE70E0AB01421B530B9B01281B77
:100FA000390B8FE391E0DC01A01BB10B8C010E1912
:100FB0001F09B801F9017D01CA0112C04FE351E0D8
:100FC000DA01A21BB30B9A01261B370BC901B90129
:100FD000F70198018C01C7017D0102C0B701FC0136
:100FE000AD8DBE8D5C9148A545234C9312B8AF8D55
:100FF000B8A15C9149A545234C93AF8DB8A15C91F4
:101000004DA1452B4C9340E542B9AF8DB8A15C9101
:1010100049A545234C93AF8DB8A15C914DA1452BBB
:101020004C93AD8DBE8D5C914CA1452B4C9392B9E8
:10103000AF8DB8A14C9199A594239C93AF8DB8A185
:101040004C919DA1942B9C9382B9AF8DB8A19C919A
:1010500089A589238C93AF8DB8A19C918DA1892BF3
:101060008C93AD8DBE8D9C9188A589238C9312B8ED
:10107000AF8DB8A19C9189A589238C93AF8DB8A120
:101080009C918DA1892B8C9381E582B9AF8DB8A1FC
:101090009C9189A589238C93AF8DB8A19C918DA13A
:1010A000892B8C93AD8DBE8D9C918CA1892B8C93BB
:1010B00032B9AF8DB8A19C9189A589238C93AF8D4E
:1010C000B8A19C918DA1892B8C9322B9AF8DB8A129
:1010D0009C9189A589238C93AF8DB8A19C918DA1FA
:1010E000892B8C93AD8DBE8D9C9188A589238C9383
:1010F00012B8AF8DB8A19C9189A589238C93AF8D2F
:10110000B8A19C918DA1892B8C9382E582B9AF8D7A
:10111000B8A19C9189A589238C93AF8DB8A19C918E
:101120008DA1892B8C93AD8DBE8D9C918CA1892B2B
:101130008C93F2B8AF8DB8A19C9189A589238C932B
:10114000AF8DB8A19C918DA1892B8C93E2B8AF8D06
:10115000B8A19C9189A589238C93AF8DB8A19C914E
:101160008DA1892B8C93AD8DBE8D9C9188A58923F3
:101170008C9312B8AF8DB8A19C9189A589238C93CB
:10118000AF8DB8A19C918DA1892B8C9383E582B9F9
:10119000AF8DB8A19C9189A589238C93AF8DB8A1FF
:1011A0009C918DA1892B8C93AD8DBE8D9C918CA132
:1011B000892B8C9312B9AF8DB8A19C9189A58923F5
:1011C0008C93AF8DB8A19C918DA1892B8C9302B982
:1011D000AF8DB8A19C9189A589238C93AF8DB8A1BF
:1011E0009C918DA1892B8C93AD8DBE8D9C9188A5F2
:1011F00089238C9312B8AF8DB8A19C9189A58923BE
:101200008C93AF8DB8A19C918DA1892B8C9380E29A
:1012100082B9AF8DB8A19C9189A589238C93AF8D9C
:10122000B8A19C918DA1892B8C93AD8DBE8D9C9185
:101230008CA1892B8C93F2B9AF8DB8A19C9189A513
:1012400089238C93AF8DB8A19C918DA1892B8C9310
:10125000E2B9EF8DF8A1908189A589238083EF8D74
:10126000F8A190818DA1892B8083ED8DFE8D9081D9
:1012700088A58923808312B8EF8DF8A1908189A574
:1012800089238083EF8DF8A190818DA1892B8083A4
:1012900081E282B9EF8DF8A1908189A589238083AD
:1012A000EF8DF8A190818DA1892B8083ED8DFE8D2E
:1012B00090818CA1892B808372B9EF8DF8A19081E8
:1012C00089A589238083EF8DF8A190818DA1892B39
:1012D000808362B92FC1413009F039C1ED8DFE8D97
:1012E000508148A54523408342E042B9EF8DF8A1E3
:1012F000508149A545234083EF8DF8A150814DA130
:10130000452B4083ED8DFE8D50814CA1452B4083B4
:1013100092B9EF8DF8A1408199A594239083EF8D28
:10132000F8A140819DA1942B9083ED8DFE8D40818D
:1013300098A59423908393E092B9EF8DF8A1408112
:1013400099A594239083EF8DF8A140819DA1942BC2
:101350009083ED8DFE8D40819CA1942B908382B96A
:10136000EF8DF8A1908189A589238083EF8DF8A165
:1013700090818DA1892B8083ED8DFE8D908188A534
:101380008923808386E082B9EF8DF8A1908189A5B9
:1013900089238083EF8DF8A190818DA1892B808393
:1013A000ED8DFE8D90818CA1892B8083F2B8EF8D1D
:1013B000F8A1908189A589238083EF8DF8A1908180
:1013C0008DA1892B8083ED8DFE8D908188A5892349
:1013D000808387E082B9EF8DF8A1908189A5892368
:1013E0008083EF8DF8A190818DA1892B8083ED8D75
:1013F000FE8D90818CA1892B8083E2B8EF8DF8A1BE
:10140000908189A589238083EF8DF8A190818DA19A
:10141000892B8083ED8DFE8D908188A58923808323
:1014200084E082B9EF8DF8A1908189A5892380831A
:10143000EF8DF8A190818DA1892B8083ED8DFE8D9C
:1014400090818CA1892B808332B9EF8DF8A1908196
:1014500089A589238083EF8DF8A190818DA1892BA7
:101460008083ED8DFE8D908188A58923808385E022
:1014700082B9EF8DF8A1908189A589238083EF8DB2
:10148000F8A190818DA1892B8083ED8DFE8D9081B7
:101490008CA1892B808322B9EF8DF8A1908189A539
:1014A00089238083EF8DF8A190818DA1892B808382
:1014B000ED8DFE8D908188A58923808388E082B997
:1014C000EF8DF8A1908189A589238083EF8DF8A104
:1014D00090818DA1892B8083ED8DFE8D90818CA1D3
:1014E000892B808312B9EF8DF8A1908189A589237A
:1014F0008083EF8DF8A190818DA1892B8083ED8D64
:10150000FE8D908188A58923808389E082B9EF8D43
:10151000F8A1908189A589238083EF8DF8A190811E
:101520008DA1892B8083ED8DFE8D90818CA1892BDF
:10153000808302B9EF8DF8A1908189A589238083EA
:10154000EF8DF8A190818DA1892B80832DC0425011
:10155000423050F5092E000CAA0BBB0BDC01992779
:101560008827A901330F660B770B9A01AB01282B53
:10157000392B4A2B5B2B6AE2CE0118D6C701FF0C30
:10158000AA0BBB0BBC0155274427012E000C220BD4
:10159000330BD901C801842B952BA62BB72B9C01AB
:1015A000AD016BE2CE0102D6EB8DFC8D90818BA15B
:1015B000892B8083DF91CF911F910F91FF90EF9046
:1015C0000895CF92DF92EF92FF920F931F93CF93E4
:1015D000DF93EC016801121613060CF04AC057FDA8
:1015E00048C08A859B85481759070CF042C0E8859A
:1015F000F9856E177F070CF03CC07901E60EF71EE7
:10160000C701019797FD35C077FF31C060E070E0FA
:101610008E179F072CF0CF0101977F01E61AF70A7A
:101620008A019C01CE018FDC9701FF0C440B550B06
:10163000B601CE018CD68A8D81110FC00A851B851B
:1016400001501109288539852150310940E050E0C9
:1016500060E070E0CE0177DC0CC0CE01DF91CF916D
:101660001F910F91FF90EF90DF90CF90B6CB790153
:10167000CFCFDF91CF911F910F91FF90EF90DF902F
:10168000CF9008950F93CF93DF9300D0CDB7DEB7FF
:101690006450643090F4E62FF0E0E85EFD4F208166
:1016A00027FD0BC029835A834B8303E09E012F5FE4
:1016B0003F4F42E068E00E940A1D0F900F900F908C
:1016C000DF91CF910F910895EF92FF920F931F93A7
:1016D000CF93DF9300D0CDB7DEB76450643010F500
:1016E000E62FF0E0E85EFD4F108117FD1BC0622F72
:1016F0009A017C01603151F0AFEFBFEF0E941A31C7
:101700002FEF30E040E050E00E94DC3019833A8354
:101710002B8303E09E012F5F3F4F41E068E0C7014C
:101720000E940A1D0F900F900F90DF91CF911F9193
:101730000F91FF90EF900895EF92FF920F931F93F8
:10174000CF93DF931F921F92CDB7DEB7633069F05E
:1017500020F4623021F540E009C0643021F06530AA
:10176000F1F443E003C042E001C041E0495F24EFEF
:10177000E22EFF24F39402E09E012F5F3F4F69E0C9
:101780000E949E1D09811A8110270127102761E000
:1017900070E080E090E00E941417C80102C080E071
:1017A00090E00F900F90DF91CF911F910F91FF90DC
:1017B000EF900895EF92FF920F931F93CF93DF93D3
:1017C000EC01F22EE32E77FDF3C157FDF1C18885C0
:1017D0009985681779070CF0EBC18A859B854817B6
:1017E00059070CF0E5C1EB8DFC8D90818FA1892309
:1017F00080838A8D8111B6C08D89823059F0833003
:10180000B1F08130D1F48FEE90E0841B950BAB01E9
:10181000BC0113C08FEE90E09C01261B370BB90171
:101820008FE391E09C01241B350BA90106C08FE3D7
:1018300091E0861B970BBA01AC01ED8DFE8D908176
:1018400088A58923808312B8EF8DF8A1908189A59E
:1018500089238083EF8DF8A190818DA1892B8083CE
:1018600080E282B9EF8DF8A1908189A589238083D8
:10187000EF8DF8A190818DA1892B8083ED8DFE8D58
:1018800090818CA1892B808372B9EF8DF8A1908112
:1018900089A589238083EF8DF8A190818DA1892B63
:1018A000808362B9EF8DF8A1908189A58923808317
:1018B000EF8DF8A190818DA1892B8083ED8DFE8D18
:1018C000908188A58923808312B8EF8DF8A190813B
:1018D00089A589238083EF8DF8A190818DA1892B23
:1018E000808381E282B9EF8DF8A1908189A5892357
:1018F0008083EF8DF8A190818DA1892B8083ED8D60
:10190000FE8D90818CA1892B808352B9EF8DF8A137
:10191000908189A589238083EF8DF8A190818DA185
:10192000892B808342B9EF8DF8A1908189A5892305
:101930008083EF8DF8A190818DA1892B8083ED8D1F
:10194000FE8D908188A58923808312B8EF8DF8A140
:10195000908189A589238083EF8DF8A190818DA145
:10196000892BD5C0813009F0D5C0ED89E150E33035
:1019700028F4F0E0E15FFD4F908101C090E0ED8D33
:10198000FE8D208188A58223808386E182B9EF8D38
:10199000F8A1208189A582238083EF8DF8A1208181
:1019A0008DA1822B8083ED8DFE8D20818CA1822BD9
:1019B000808392B9EF8DF8A1908189A589238083D6
:1019C000EF8DF8A190818DA1892B8083ED8DFE8D07
:1019D000908188A58923808382E082B9EF8DF8A168
:1019E000908189A589238083EF8DF8A190818DA1B5
:1019F000892B8083ED8DFE8D90818CA1892B808336
:101A000072B9EF8DF8A1908189A589238083EF8D2C
:101A1000F8A190818DA1892B8083ED8DFE8D908121
:101A200088A58923808383E082B9EF8DF8A1908116
:101A300089A589238083EF8DF8A190818DA1892BC1
:101A40008083ED8DFE8D90818CA1892B808362B97E
:101A5000EF8DF8A1908189A589238083EF8DF8A16E
:101A600090818DA1892B8083ED8DFE8D908188A53D
:101A70008923808386E082B9EF8DF8A1908189A5C2
:101A800089238083EF8DF8A190818DA1892B80839C
:101A9000ED8DFE8D90818CA1892B808352B9EF8DC5
:101AA000F8A1908189A589238083EF8DF8A1908189
:101AB0008DA1892B8083ED8DFE8D908188A5892352
:101AC000808387E082B9EF8DF8A1908189A5892371
:101AD0008083EF8DF8A190818DA1892B8083ED8D7E
:101AE000FE8D90818CA1892B808342B9EF8DF8A166
:101AF000908189A589238083EF8DF8A190818DA1A4
:101B0000892B8083ED8DFE8D908188A5892380832C
:101B100082E21BC08250823008F044C00A851B85D7
:101B2000015011092885398521503109CE010BDA80
:101B3000EB8DFC8D90818FA189238083ED8DFE8DAF
:101B4000908188A5892380838CE282B9EF8DF8A1EA
:101B5000908189A589238083EF8DF8A190818DA143
:101B6000892B8083ED8DFE8D90818CA1892B8083C4
:101B7000E2B8EF8DF8A1908189A589238083EF8D4C
:101B8000F8A190818DA1892B8083F2B8EF8DF8A107
:101B9000908189A589238083EF8DF8A190818DA103
:101BA000892B8083EB8DFC8D90818BA1892B808389
:101BB000DF91CF911F910F91FF90EF900895EF92D9
:101BC000FF920F931F93CF93DF93EC010E94460483
:101BD000EB8DFC8D90818FA1892380838A8D81116B
:101BE0005CC0ED89E150E33038F4F0E0EE0FFF1F08
:101BF000EE5EFD4F908101C090E3ED8DFE8D208162
:101C000088A58223808312B8EF8DF8A1208189A551
:101C100082238083EF8DF8A120818DA1822B808388
:101C200083E082B9EF8DF8A1208189A5822380838A
:101C3000EF8DF8A120818DA1822B8083ED8DFE8D0B
:101C400020818CA1822B808380E182B9EF8DF8A165
:101C5000208189A582238083EF8DF8A120818DA129
:101C6000822B808392B9EF8DF8A1908189A5892379
:101C70008083EF8DF8A190818DA1892B80830A85C7
:101C80001B8501501109288539852150310940E013
:101C900050E060E070E0CE0156D98A8D813099F530
:101CA000ED89E150E33028F4F0E0E15FFD4F9081F1
:101CB00001C090E0ED8DFE8D208188A58223808378
:101CC00086E182B9EF8DF8A1208189A582238083E6
:101CD000EF8DF8A120818DA1822B8083ED8DFE8D6B
:101CE00020818CA1822B808392B9EF8DF8A1908105
:101CF00089A589238083EF8DF8A190818DA1892BFF
:101D00008083CE016AD88A8D823009F048C08D89DF
:101D1000813071F050F0823029F0833059F458E26C
:101D2000E52E08C068E4E62E05C048E8E42E02C0AF
:101D300038EEE32EED8DFE8D908188A5892380837A
:101D400086E382B9EF8DF8A1908189A589238083EC
:101D5000EF8DF8A190818DA1892B8083ED8DFE8D73
:101D600090818CA1892B8083E2B8EF8DF8A19081BE
:101D700089A589238083EF8DF8A190818DA1892B7E
:101D800080830A851B8501501109288539852150DA
:101D9000310940E050E060E070E0CE01D4D88A8D97
:101DA000833009F047C08D89813069F048F0823076
:101DB00029F0833051F420E6F22E07C0F12C05C043
:101DC00090ECF92E02C080EAF82EED8DFE8D908108
:101DD00088A58923808386E382B9EF8DF8A190815D
:101DE00089A589238083EF8DF8A190818DA1892B0E
:101DF0008083ED8DFE8D90818CA1892B8083F2B83C
:101E0000EF8DF8A1908189A589238083EF8DF8A1BA
:101E100090818DA1892B80830A851B850150110932
:101E2000288539852150310940E050E060E070E0BC
:101E3000CE0189D8DF91CF911F910F91FF90EF9044
:101E40000895EF92FF920F931F93CF93DF93EC01CE
:101E50007B018A8D81119DC0ED89E150E33060F4F2
:101E6000F0E0DF01A45FBD4F8C91EE0FFF1FEA5F32
:101E7000FD4F2081318104C020E030E080E090E01F
:101E8000EB8DFC8D40819FA194239083ED8DFE8D81
:101E9000408198A59423908312B8EF8DF8A14081DA
:101EA00099A594239083EF8DF8A140819DA1942B57
:101EB000908390E292B9EF8DF8A1408199A5942387
:101EC0009083EF8DF8A140819DA1942B9083ED8D9F
:101ED000FE8D40819CA1942B908312B8EF8DF8A1C8
:101EE000408199A594239083EF8DF8A140819DA115
:101EF000942B908382B9EF8DF8A1908189A58923D5
:101F00008083EF8DF8A190818DA1892B8083ED8D49
:101F1000FE8D908188A58923808312B8EF8DF8A16A
:101F2000908189A589238083EF8DF8A190818DA16F
:101F3000892B808381E282B9EF8DF8A1908189A5F8
:101F400089238083EF8DF8A190818DA1892B8083D7
:101F5000ED8DFE8D90818CA1892B808332B9EF8D20
:101F6000F8A1908189A589238083EF8DF8A19081C4
:101F70008DA1892B808322B9EF8DF8A1908189A54D
:101F800089238083EF8DF8A190818DA1892B808397
:101F900012C08150833078F40A851B8501501109E5
:101FA000288539852150310940E050E060E070E03B
:101FB000CE010E94A30720E03CE241E050E0B701DF
:101FC000CE01DF91CF911F910F91FF90EF90BFC194
:101FD0008F929F92AF92BF92CF92DF92EF92FF9239
:101FE0000F931F93CF93DF93EC0147011216130653
:101FF0000CF06AC0101611060CF066C0A885B985F1
:102000006A177B070CF060C0CA84DB844C155D0541
:102010000CF05AC07901E60EF71EC701019797FD33
:1020200053C05801A40EB51EF5013197F7FD4CC001
:1020300077FF48C060E070E057FD02C0580102C061
:1020400040E050E08A179B072CF0CD0101977D01FD
:10205000E61AF70AEC15FD052CF0F601319756014A
:10206000A41AB50A8F019C01CE010E94A307970113
:10207000D5010E9419329B01AC01B401CE0167D198
:102080008A8D811110C00A851B8501501109288590
:1020900039852150310940E050E060E070E0CE0128
:1020A0000E94A30711C0CE01DF91CF911F910F9124
:1020B000FF90EF90DF90CF90BF90AF909F908F9068
:1020C0000C94ED067901B8CFDF91CF911F910F915C
:1020D000FF90EF90DF90CF90BF90AF909F908F9048
:1020E0000895CF92DF92EF92FF920F931F93CF93B9
:1020F000DF93EC016801121613060CF04EC077FD59
:102100004CC088859985681779070CF046C08A8588
:102110009B85481759070CF040C07901E40EF51E65
:1021200087010150110917FD38C057FF34C040E046
:1021300050E00817190734F08C01015011097C0197
:10214000E41AF50A9B01CE010E94A3079701FF0C38
:10215000440B550BB601CE01FAD08A8D811110C007
:102160000A851B85015011092885398521503109BF
:1021700040E050E060E070E0CE010E94A3070DC097
:10218000CE01DF91CF911F910F91FF90EF90DF90E3
:10219000CF900C94ED067901CCCFDF91CF911F91B8
:1021A0000F91FF90EF90DF90CF900895CF92DF9244
:1021B000EF92FF92FC01A38DB48D9C9187A189239E
:1021C0008C93A58DB68D9C9180A589238C9362B943
:1021D000A78DB0A19C9181A589238C93A78DB0A1D7
:1021E0009C9185A1892B8C93A58DB68D9C9184A102
:1021F000892B8C9383E290E0DC011197F1F7C52ED7
:10220000DD24EE24FF24C2B8A78DB0A17C9161A586
:1022100067236C93A78DB0A17C9165A1672B6C930C
:10222000DC011197F1F76A01EE24FF24C2B8A78DF3
:10223000B0A17C9161A567236C93A78DB0A17C911F
:1022400065A1672B6C93DC011197F1F7C32ED42E97
:10225000E52EFF24C2B8A78DB0A17C9161A56723AC
:102260006C93A78DB0A17C9165A1672B6C930197AE
:10227000F1F722B9A78DB0A19C9181A589238C93F8
:10228000A78DB0A19C9185A1892B8C93A38DB48D32
:102290009C9183A1892B8C93FF90EF90DF90CF903E
:1022A000089590E0FC013197E231F10508F04EC04D
:1022B0008827EE58FF4F8F4F0C940A328091800090
:1022C0008F7703C0809180008F7D80938000089578
:1022D00080918000877FF9CF84B58F7702C084B565
:1022E0008F7D84BD08958091B0008F7703C0809169
:1022F000B0008F7D8093B0000895809190008F771B
:1023000007C0809190008F7D03C080919000877FEF
:102310008093900008958091A0008F7707C08091EE
:10232000A0008F7D03C08091A000877F8093A000D4
:102330000895809120018F7707C0809120018F7DC3
:1023400003C080912001877F8093200108951F930F
:10235000CF93DF93FC01A38DB48D9C9187A189233A
:102360008C93A58DB68D9C9180A589238C93828DAD
:10237000823091F081110EC012B8A78DB0A19C914E
:1023800081A589238C93A78DB0A19C9185A1892BD0
:102390008C9304C0833011F48CE201C082E282B9D4
:1023A000A78DB0A19C9181A589238C93A78DB0A105
:1023B0009C9185A1892B8C93A58DB68D9C9184A130
:1023C000892B8C9372B9A78DB0A19C9181A589238B
:1023D0008C93A78DB0A19C9185A1892B8C9362B918
:1023E000A78DB0A19C9181A589238C93A78DB0A1C5
:1023F0009C9185A1892B8C93215031094109510968
:10240000DA01C90136E0B695A795979587953A9573
:10241000D1F77613F0C0019708F465C060E1A78D8D
:10242000B0A1CC9171A57C237C93A78DB0A1CC9158
:1024300075A17C2B7C93A78DB0A1CC9171A57C2339
:102440007C93A78DB0A1CC9175A17C2B7C93A78D9B
:10245000B0A1CC9171A57C237C93A78DB0A1CC9128
:1024600075A17C2B7C93A78DB0A1CC9171A57C2309
:102470007C93A78DB0A1CC9175A17C2B7C93A78D6B
:10248000B0A1CC9171A57C237C93A78DB0A1CC91F8
:1024900075A17C2B7C93A78DB0A1CC9171A57C23D9
:1024A0007C93A78DB0A1CC9175A17C2B7C93A78D3B
:1024B000B0A1CC9171A57C237C93A78DB0A1CC91C8
:1024C00075A17C2B7C93A78DB0A1CC9171A57C23A9
:1024D0007C93A78DB0A1CC9175A17C2B7C9361508E
:1024E00009F09DCF98CF2F73215008F4A6C0A78D77
:1024F000B0A19C9181A589238C93A78DB0A19C91BB
:1025000085A1892B8C93A78DB0A19C9181A589234E
:102510008C93A78DB0A19C9185A1892B8C93E4CF3E
:1025200072B9C78DD0A11881B1A5B123B883C78D69
:10253000D0A11881B5A1B12BB88362B9C78DD0A144
:102540001881B1A5B123B883C78DD0A11881B5A1D9
:10255000B12BB88372B9C78DD0A11881B1A5B123B1
:10256000B883C78DD0A11881B5A1B12BB88362B94A
:10257000C78DD0A11881B1A5B123B883C78DD0A1D3
:102580001881B5A1B12BB88372B9C78DD0A11881BC
:10259000B1A5B123B883C78DD0A11881B5A1B12B46
:1025A000B88362B9C78DD0A11881B1A5B123B88312
:1025B000C78DD0A11881B5A1B12BB88372B9C78DD1
:1025C000D0A11881B1A5B123B883C78DD0A118813E
:1025D000B5A1B12BB88362B9C78DD0A11881B1A5BF
:1025E000B123B883C78DD0A11881B5A1B12BB88311
:1025F000A15009F095CF019710F0A0E191CF2F7372
:102600002150D8F072B9A78DB0A19C9181A58923E2
:102610008C93A78DB0A19C9185A1892B8C9362B9D5
:10262000A78DB0A19C9181A589238C93A78DB0A182
:102630009C9185A1892B8C93E3CFA38DB48D9C9124
:1026400083A1892B8C93DF91CF911F910895FC0179
:1026500044815581608171818DE497E03AC7CF93C1
:10266000DF93EC0141E050E065EE74E032D7811178
:1026700002C0CE018BD7CE01DF91CF9108956115B5
:10268000710549F0FB0101900020E9F73197AF0196
:10269000461B570B1EC780E00895EF92FF920F93E1
:1026A0001F93CF93DF93CDB7DEB728970FB6F8947B
:1026B000DEBF0FBECDBF7C01CB014AE08E010F5FB4
:1026C0001F4FB8010E94422DF80101900020E9F748
:1026D0003197AF01401B510BB801C701FAD62896BC
:1026E0000FB6F894DEBF0FBECDBFDF91CF911F9123
:1026F0000F91FF90EF900895282F30913A063132D4
:1027000008F04AC0809116068111FCCF90913906DD
:1027100042E040931606209315062FEF20931406EF
:102720001092130630931206E9E1F6E0A2EFB5E04D
:1027300020E0321721F041914D932F5FFACF109294
:10274000F1052091F105990F922B9093F10590914D
:10275000F005913061F41092F0059091F10590939D
:10276000BB009091BC0093FDF8CF95EC01C095EEB5
:102770009093BC00909116069230E1F3909114066C
:102780009F3F79F080911406803241F080911406C9
:10279000803331F084E005C081E003C082E001C0F5
:1027A00083E01092180610923A06109217060895C8
:1027B000EF92FF920F93CF93DF9300D01F92CDB78C
:1027C000DEB728EEE22E23E0F22E04E09E012F5F1A
:1027D0003F4F44E060E00E949E1D69817A818B81B9
:1027E0009C810E9412320E94C92F20E030E040E814
:1027F00057E30E9428300F900F900F900F90DF91B9
:10280000CF910F91FF90EF900895EF92FF920F9369
:10281000CF93DF9300D01F92CDB7DEB72DE7E22E26
:10282000F12C04E09E012F5F3F4F42E060E00E94E8
:102830009E1D69817A818B819C810E9412320F904A
:102840000F900F900F90DF91CF910F91FF90EF902D
:1028500008952FB7F8948091E6059091E705A0912F
:10286000E805B091E9052FBF8093A6069093A706CF
:10287000A093A806B093A9068EE996E049D497FFE5
:1028800026C02FB7F8948091E6059091E705A091B6
:10289000E805B091E9052FBF4091A6065091A70623
:1028A0006091A8067091A906841B950BA60BB70B27
:1028B0004091A2065091A3066091A4067091A506CE
:1028C00084179507A607B707B8F28FEF9FEF089513
:1028D0002F923F924F925F926F927F928F929F9230
:1028E000AF92BF92CF92DF92EF92FF920F931F931E
:1028F000CF93DF93CDB7DEB76B970FB6F894DEBFFB
:102900000FBECDBF9B8F8A8F5B011A01D22E1F8312
:102910000E833701C982DC0158962D913C9159975D
:102920002115310509F0E6C018968D919C911997F3
:10293000681779070CF0CDC11A968D919C911B9761
:10294000481759070CF0C5C18C2C912CFB0126E0CF
:10295000C29EE00DF11D1124FB87EA871E161F069B
:102960000CF0B7C1A40183E0440F551F8A95E1F72D
:102970005D874C87CA01820D931D181619060CF04D
:10298000A8C157968C91811104C05FEA5D1508F4C7
:10299000D394AA8DBB8DED91FC9111970284F385A0
:1029A000E02DCD011995B5E0DB9EC0011124F501A4
:1029B0003596FF87EE87BB82AA8225019C012A19E2
:1029C0003B09398B288BA101485F5F4F5B8B4A8B9A
:1029D000E889F989E40DF51DE458FD4F54915887B5
:1029E00061013D822C82888580FF13C0AA8DBB8D3A
:1029F000ED91FC91B981B13031F40484F585E02D7D
:102A00002E813F8116C00684F785E02DEE80FF8081
:102A10001AC0EE81FF81E615F705F1F0AA8DBB8D96
:102A2000ED91FC91B981B13051F40484F585E02D2C
:102A30009301A601B2018A8D9B8D19950DC0068464
:102A4000F785E02D7301840194014C815D816A81D9
:102A50007B818A8D9B8D1995E885E695E887FFEF48
:102A6000CF1ADF0A2C813D81280D391D3D832C832F
:102A70004A895B89C416D50609F0B5CF5FEF451AC0
:102A8000550A8A819B81880D991D9B838A83AE8517
:102A9000BF854A165B0609F09BCFEE81FF81E615E4
:102AA000F70509F4F4C0EA8DFB8DA081B181F981AD
:102AB000F13079F4B5016B5F7F4F5096ED91FC9149
:102AC0005197830128E030E0A1018A8D9B8D1995F3
:102AD000DEC06A857B85681979091E96ED91FC91A7
:102AE0001F9773010C851D859401A1018A8D9B8D13
:102AF0001995CDC0F9013496E491DE1AF9013296A8
:102B000085919491B7E0DB9E800D911D1124F90110
:102B1000259134913B8B2A8BFC012591349129011D
:102B2000FC013296C490319634913E8732961491CE
:102B30003196D4904981423058F0612E012E000C1C
:102B400077088D2D0D2C000C990B9987888704C070
:102B500019861886612C712CAA8DBB8DED91FC9184
:102B600011970284F385E02DCD011995B9818B2E43
:102B7000912C689CC001699C900D789C900D11244B
:102B8000FC01EA0DFB1DFD87EC871A82712C612C7C
:102B9000E12F110FFF0B95012E0F3F1F3B872A8757
:102BA000AC0CB11CA5014E0F5F1F5F8B4E8BC1019A
:102BB0008D0D911DD7FC9A95998F888F9E856916EA
:102BC00008F065C0862D90E048855985480F591F4B
:102BD000489D9001499D300D589D300D1124D10123
:102BE000A20FB31FB98BA88BEC85FD85FD83EC8309
:102BF000AA84BB84DA80FA85DF1A288D398D280FE4
:102C0000391F3D8B2C8B8D2D8A0D4E895F89A41623
:102C1000B506C1F1877041F4C2010196EA89FB89CA
:102C2000E40DF51D74902C0177FE21C0AA8DBB8D9B
:102C3000ED91FC91B981B13061F40484F585E02D0A
:102C40002E813F814C895D89B5018A8D9B8D1995B7
:102C50000EC00684F785E02DEE80FF80840194018C
:102C6000488959896C817D818A8D9B8D1995770C56
:102C7000EFEFAE1ABE0A2C813D81280D391D3D8330
:102C80002C83C1CF3A813C0D3A83639497CFAA8DB0
:102C9000BB8DED91FC9111970688F789E02DCD0150
:102CA0006B960FB6F894DEBF0FBECDBFDF91CF910C
:102CB0001F910F91FF90EF90DF90CF90BF90AF905A
:102CC0009F908F907F906F905F904F903F902F904C
:102CD00019946B960FB6F894DEBF0FBECDBFDF918F
:102CE000CF911F910F91FF90EF90DF90CF90BF9009
:102CF000AF909F908F907F906F905F904F903F909C
:102D00002F900895CF93DF93282F30E0F901EA5CEC
:102D1000FD4F8491F901E458F84FD491F901E45240
:102D2000F84FC491CC2389F08111BBDAEC2FF0E08D
:102D3000EE0FFF1FE45EFD4FA591B491EC91ED23E2
:102D400081E090E021F480E002C080E090E0DF913B
:102D5000CF9108951F93CF93DF93282F30E0F9018F
:102D6000EA5CFD4F8491F901E458F84FD491F901E0
:102D7000E452F84FC491CC23B9F0162F811191DAA7
:102D8000EC2FF0E0EE0FFF1FEE53F84FA591B4913A
:102D90009FB7F894111104C08C91D095D82302C02C
:102DA000EC91DE2BDC939FBFDF91CF911F910895B3
:102DB000CF93DF9390E0FC01E458F84F2491FC019D
:102DC000E452F84F8491882361F190E0880F991FB5
:102DD000FC01EE5FFD4FC591D491FC01EE53F84F1D
:102DE000A591B491611109C09FB7F894888120958D
:102DF00082238883EC912E230BC0623061F49FB74D
:102E0000F8948881322F309583238883EC912E2B80
:102E10002C939FBF06C08FB7F894E8812E2B288390
:102E20008FBFDF91CF9108958F929F92AF92BF9203
:102E3000CF92DF92EF92FF926B017C010E94C2233E
:102E40004B015C01C114D104E104F104F1F00E94D2
:102E5000C223DC01CB0188199909AA09BB09883E64
:102E60009340A105B10570F321E0C21AD108E10831
:102E7000F10888EE880E83E0981EA11CB11CC114D5
:102E8000D104E104F10419F7DDCFFF90EF90DF905A
:102E9000CF90BF90AF909F908F900895EF92FF9248
:102EA0000F931F93CF93DF931F921F92CDB7DEB77F
:102EB00028EEE22E23E0F22E02E09E012F5F3F4F2C
:102EC00040E16FE03BD609811A81102701271027C6
:102ED00061E070E080E090E0A7DFC8010F900F9004
:102EE000DF91CF911F910F91FF90EF900895CF92B6
:102EF000DF92EF92FF920F931F93CF93DF931F9276
:102F00001F92CDB7DEB76C01FC0164831FEF1783FE
:102F10001092EF051092EE051092180610923A06E4
:102F20001092160681E0809315061092F00561E07C
:102F300084E110DF61E085E10DDF8091B9008E7FD3
:102F40008093B9008091B9008D7F8093B90088E4A7
:102F50008093B80085E48093BC0088EB99E190935E
:102F6000ED058093EC0589EB99E19093EB05809357
:102F7000EA051A8301E09E012E5F3F4F4FE760E0B4
:102F8000C60148D564EF71E080E090E04DDF8DE749
:102F9000E82EF12C9E012F5F3F4F41E060E0C6011B
:102FA000CDD5998181E0953509F080E00F900F90A3
:102FB000DF91CF911F910F91FF90EF90DF90CF9015
:102FC0000895E0918207F0918307908180918A07AC
:102FD000892B8083E0918607F0918707908180910B
:102FE0008C07892B8083E0918807F0918907908175
:102FF00080918D07892B808380919207882359F0D7
:1030000060E0A8DE62E070E080E090E00DDF61E06B
:10301000809192079FDEE0918207F0918307908173
:1030200080918E0789238083E0918407F091850742
:10303000908180918F078923808312B8E091860761
:10304000F091870790818091900789238083E09198
:103050008607F0918707908180918C07892B808368
:1030600083E0E0918607F091870720819091900797
:1030700092239083E0918607F091870720819091B9
:103080008C07922B9083815061F7E0918207F09139
:103090008307908180918A07892B80830895CF923E
:1030A000DF92EF92FF920F931F93CF93DF936C0108
:1030B0007A018B01C0E0D0E0CE15DF0581F0D801A8
:1030C0006D918D01D601ED91FC910190F081E02D83
:1030D000C6011995892B11F02196EECF7E01C7010B
:1030E000DF91CF911F910F91FF90EF90DF90CF90E4
:1030F0000895FC01538D448D252F30E0842F90E0FE
:10310000821B930B541710F0CF96089501970895E2
:10311000FC01918D828D981761F0828DDF01A80FDF
:10312000B11D5D968C91928D9F5F9F73928F90E001
:1031300008958FEF9FEF0895FC01918D828D981770
:1031400031F0828DE80FF11D858D90E008958FEFAD
:103150009FEF0895FC01918D228D892F90E0805C76
:103160009F4F821B91098F73992708958EE996E0EE
:10317000F1DF21E0892B09F420E0822F0895FC0182
:10318000848DDF01A80FB11DA35ABF4F2C91848DF0
:1031900090E001968F739927848FA689B7892C9325
:1031A000A089B1898C91837080648C93938D848D78
:1031B000981306C00288F389E02D80818F7D80837B
:1031C0000895EF92FF920F931F93CF93DF93EC013B
:1031D00081E0888F9B8D8C8D981305C0E889F989D3
:1031E000808185FD25C0F62E0B8D10E00F5F1F4FEF
:1031F0000F731127E02E8C8DE8120BC00FB607FC61
:10320000FACFE889F989808185FFF5CFCE01B7DF54
:10321000F2CF8B8DFE01E80FF11DE35AFF4FF082D4
:103220009FB7F8940B8FEA89FB89808180620AC07E
:103230009FB7F894EE89FF896083E889F9898081D6
:103240008370806480839FBF81E090E0DF91CF91A5
:103250001F910F91FF90EF900895CF93DF93EC01B2
:10326000888D8823C1F0EA89FB89808185FD05C0AE
:10327000A889B9898C9186FD0EC00FB607FCF5CFE1
:10328000808185FFF2CFA889B9898C9185FFEDCF28
:10329000CE0175DFE8CFDF91CF91089580E090E017
:1032A000892B19F063DF811125C080E090E0892B24
:1032B00041F080E090E0892B21F00E940000811114
:1032C0001CC080E090E0892B41F080E090E0892BE9
:1032D00021F00E940000811113C080E090E0892B52
:1032E000A1F080E090E0892B81F00E940000811124
:1032F0000AC008950E940000D8CF0E940000E1CFCC
:103300000E940000EACF0C940000089585ED8093A0
:10331000BC008091BC0084FDFCCF1092160608957D
:1033200040917B06262F30E0240F311D21323105DC
:10333000DCF4209116062430C9F4FC0180E090E012
:10334000861758F430917B062191DC01A55AB94FBC
:10335000A30FB11D2C930196F3CF80917B06680FCC
:1033600060937B0680E0089581E0089582E00895EF
:10337000089508950895E091EF058091EE05E8170E
:1033800030F4F0E0E55CF94F808190E008958FEF34
:103390009FEF08959091EF058091EE05981750F4F6
:1033A000E92FF0E0E55CF94F208130E09F5F9093DA
:1033B000EF0502C02FEF3FEFC90108958091EE05A0
:1033C00090E02091EF05821B91090895CF92DF9242
:1033D000EF92FF920F931F93CF93DF937C01CB016A
:1033E0008A0120911706222389F0EB016B01C40E9C
:1033F000D51ECC15DD0561F06991D701ED91FC91E9
:103400000190F081E02DC7011995F3CF642F88DF7B
:10341000C801DF91CF911F910F91FF90EF90DF9046
:10342000CF900895CF93DF931F92CDB7DEB7698316
:10343000209117062223D1F020913A06203240F045
:1034400021E030E0FC013383228380E090E014C06F
:1034500080911806E82FF0E0E75EF94F998190839C
:103460008F5F8093180680933A0604C061E0CE0116
:10347000019656DF81E090E00F90DF91CF910895A3
:103480000E9426340F931F93CF93DF93EC01888122
:103490009981009729F02A813B812617370788F404
:1034A0008B016F5F7F4F0E944633009761F09983D5
:1034B00088831B830A832C813D81232B11F4FC011B
:1034C000108281E001C080E0DF91CF911F910F91C8
:1034D0000895EF92FF920F931F93CF93DF9361159F
:1034E000710511F480E01BC041155105B9F07B0155
:1034F000EC018C819D818A01080F191FB801CE0152
:10350000C1DF882379F3288139818C819D81B701BE
:10351000820F931F0E943C341D830C8381E0DF9156
:10352000CF911F910F91FF90EF900895EF92FF922E
:103530000F931F93CF93DF93CDB7DEB764970FB68A
:10354000F894DEBF0FBECDBF7C01CB01BA018E0166
:103550000F5F1F4F22E044E00E94232DFC010190E9
:103560000020E9F73197AF01481B590BBC01C70197
:10357000B0DF64960FB6F894DEBF0FBECDBFDF910B
:10358000CF911F910F91FF90EF900895CF93DF930C
:10359000EC0188819981009711F00E94BD32198257
:1035A00018821D821C821B821A82DF91CF9108959E
:1035B000EF92FF920F931F93CF93DF93EC017B0168
:1035C0008A01BA015FDF811103C0CE01DFDF07C0CE
:1035D0001D830C83B701888199810E943C34CE0100
:1035E000DF91CF911F910F91FF90EF900895FC0113
:1035F000808191810C94BD32FB01DC0111961C92FB
:103600001E9213961C921E92129715961C921E9251
:1036100014978617970741F06081718161157105D4
:1036200019F044815581C4CF0895FC0111821082A4
:1036300013821282158214826115710549F0FB0113
:1036400001900020E9F73197AF01461B570BB0CF2F
:103650000895BF92CF92DF92EF92FF920F931F9344
:10366000CF93DF937C016B01EA01890124173507B1
:1036700020F48D2FE901042F182F69EC72E0C701A7
:10368000D4DFD60114968D919C911597C817D90750
:1036900030F58017910708F48C01D601ED91FC916B
:1036A0001197E00FF11FB08010826D917C916C0F2B
:1036B0007D1F6115710559F0FB0101900020E9F7AC
:1036C0003197AF01461B570BC70172DF02C0C7011C
:1036D0005DDFD601ED91FC91E00FF11FB082C701D3
:1036E000DF91CF911F910F91FF90EF90DF90CF90DE
:1036F000BF9008951F920F920FB60F9211240BB630
:103700000F922F933F934F935F936F937F938F937A
:103710009F93AF93BF93EF93FF938EE996E02FDDD6
:10372000FF91EF91BF91AF919F918F917F916F9199
:103730005F914F913F912F910F900BBE0F900FBE55
:103740000F901F9018951F920F920FB60F92112491
:103750000BB60F922F938F939F93EF93FF93E0916C
:10376000AE06F091AF068081E091B406F091B50607
:1037700082FD12C090818091B7068F5F8F73209178
:10378000B806821751F0E091B706F0E0E256F94F23
:10379000958F8093B70601C08081FF91EF919F9133
:1037A0008F912F910F900BBE0F900FBE0F901F9017
:1037B00018951F920F920FB60F9211240BB60F920D
:1037C0002F933F934F935F936F937F938F939F9329
:1037D000AF93BF93EF93FF938091B900887F8036BA
:1037E00009F49CC068F5883209F45BC090F480311C
:1037F00009F454C038F4882309F4F6C0883009F479
:103800004DC0F5C0883109F44CC0803209F45DC068
:10381000EEC0803409F468C048F4803309F455C020
:10382000883309F0E4C080931406D8C0803509F4C9
:103830004FC0883509F45DC0883409F0D8C0D6C0BF
:10384000883909F4C7C0A8F4883709F467C038F488
:10385000883609F463C0803709F460C0C8C088386E
:1038600009F4B8C0803909F45FC0803809F0BFC0DE
:103870005BC0803B09F486C038F4803A09F466C026
:10388000883A09F47FC0B3C0803C09F4A7C0883CE3
:1038900009F4A4C0883B09F48AC0A9C08091F1054D
:1038A00010C09091130680911206981770F5E09160
:1038B000130681E08E0F80931306F0E0EE50FA4F6E
:1038C00080818093BB0085EC86C0809314068EC0F7
:1038D000E091130681E08E0F809313068091BB0068
:1038E000F0E0EE50FA4F808390911306809112061B
:1038F0006EC0E091130681E08E0F809313068091D5
:10390000BB00F0E0EE50FA4F8083809115068111E4
:103910006DC081E08093F00584EA61C083E080930C
:10392000160610929D06CFCF80919D06803208F03A
:1039300051C0E0919D0681E08E0F80939D0680919D
:10394000BB00F0E0E358F94F8083BDCF85EC809356
:10395000BC001092160680919D06803230F4E091F2
:103960009D06F0E0E358F94F108260919D0670E0EB
:10397000E091EA05F091EB058DE796E0199510923C
:103980009D0635C084E08093160610927C06109246
:103990007B06E091EC05F091ED05199580917B0691
:1039A000811105C081E080937B0610925B06E09157
:1039B0007C0681E08E0F80937C06F0E0E55AF94F9B
:1039C00080818093BB0090917C0680917B06981744
:1039D00008F479CF85E88093BC0009C085EC80931A
:1039E000BC001092160603C0109214068FDCFF91E3
:1039F000EF91BF91AF919F918F917F916F915F9167
:103A00004F913F912F910F900BBE0F900FBE0F90D3
:103A10001F901895EF92FF920F931F93CF93DF9310
:103A2000EC01142F79018C8191E09093170680931B
:103A300039061092180610923A068D819E81DC019B
:103A4000ED91FC910190F081E02D19958D819E8181
:103A5000DC01ED91FC910190F081E02D612F199531
:103A60008D819E81402F50E0DC01ED91FC91028020
:103A7000F381E02DB70119958F818F3F49F481E0E3
:103A8000DF91CF911F910F91FF90EF900C947C13D9
:103A90008F8138D9892BE1F3F2CFCF92DF92EF9269
:103AA000FF920F93CF93DF93CDB7DEB7A0970FB6FA
:103AB000F894DEBF0FBECDBF6C01862FFB010E2F29
:103AC000081B9191E02EF12C992341F0A1E0B0E088
:103AD000AC0FBD1FAE0DBF1D9C93F1CF9E012F5F9C
:103AE0003F4F45E062E0C60195DFC701A0960FB6E3
:103AF000F894DEBF0FBECDBFDF91CF910F91FF9045
:103B0000EF90DF90CF9008950F93CF93DF931F92A4
:103B1000CDB7DEB7698301E09E012F5F3F4F45E0DF
:103B200062E078DF61E070E080E090E07DD981E0E4
:103B300090E00F90DF91CF910F9108952F923F92D7
:103B40004F925F926F927F928F929F92AF92BF92AD
:103B5000CF92DF92EF92FF920F931F93CF93DF9359
:103B600000D01F921F92CDB7DEB79D838C83162F96
:103B70004B8329014701880C991C880C991C25E06E
:103B8000821A9108312C22242394602E712C301635
:103B900008F0C1C0AC81BD8114968C91149720921D
:103BA0001706809339061092180610923A06159659
:103BB0008D919C911697DC01ED91FC910190F08123
:103BC000E02D612F1995EC81FD8185819681DC01C5
:103BD000ED91FC910190F081E02D6B811995EC81C4
:103BE000FD8187818F3F59F481E00E947C13F2E0D0
:103BF000EF16F10460F0C4010197F1F708C0AC8141
:103C0000BD8117968C917ED8892BC9F3EDCFEC81BD
:103C1000FD8187818F3F39F0AC81BD8117968C91F2
:103C200071D8892BC9F3809116068111FCCF9301BD
:103C3000231931092132310514F020E230E0EC8102
:103C4000FD819481822F213208F080E220921606B5
:103C500020921506FFEFF0931406109213064FEF13
:103C6000480F409312062092F1054091F105990FFB
:103C7000942B9093F1059091F005913071F410928E
:103C8000F0059091F1059093BB009091BC0093FDDD
:103C9000F8CF45EC4093BC0003C095EE9093BC0078
:103CA000909116069130E1F390911306981710F455
:103CB00080911306E2EFF5E0ABE3B6E090E09817F1
:103CC00021F041914D939F5FFACF1092EF059093B1
:103CD000EE05A12CB12C6901DD24832D8A0DAC14D5
:103CE000BD0414F0382E53CFD201A80FB11DBA83F2
:103CF000A983EC81FD8185819681DC01ED91FC91A8
:103D00000284F385E02D1995E981FA818083FFEF24
:103D1000AF1ABF0AE2CF0F900F900F900F900F9045
:103D2000DF91CF911F910F91FF90EF90DF90CF9097
:103D3000BF90AF909F908F907F906F905F904F90CB
:103D40003F902F9008950F931F93DC01ED91FC910C
:103D5000048CF58DE02D19951F910F910895DC01CC
:103D6000ED91FC910084F185E02D19942F923F9202
:103D70004F925F926F927F928F929F92AF92BF927B
:103D8000CF92DF92EF92FF920F931F93CF93DF9327
:103D900000D000D0CDB7DEB72C017E836D836A01E1
:103DA0005901C801FC82EB824801841A950A97FEEA
:103DB00003C091948194910835012D813E81621A4E
:103DC000730A77FE03C071946194710868147904D2
:103DD0005CF43A2D2B2D5C01832F922F3D812E8197
:103DE000DE82CD82C32ED22EAD81BE81AA16BB0645
:103DF0005CF43C2D2D2D6C01832F922F3D812E8163
:103E0000BE82AD82A32EB22E85012D813E81021B82
:103E1000130B1C012C183D0837FE03C0319421946C
:103E20003108780117FF03C03FEFE31AF30AF59456
:103E3000E794C816D9062CF08FEF9FEF9A838983F9
:103E400004C0A1E0B0E0BA83A9832D813E81A2160F
:103E5000B30624F1D201ED91FC910484F585E02DA7
:103E60002B813C816814790424F44D815E81B60174
:103E700003C0A6016D817E81C2011995E218F30885
:103E8000F7FE06C029813A81C20ED31EE00EF11E54
:103E90008D819E8101969E838D83D7CF26960FB606
:103EA000F894DEBF0FBECDBFDF91CF911F910F9170
:103EB000FF90EF90DF90CF90BF90AF909F908F904A
:103EC0007F906F905F904F903F902F90089508954E
:103ED00080E090E008951F920F920FB60F92112488
:103EE0008F930FB6F894A8958091600088618093B5
:103EF0006000109260000FBE8F910F900FBE0F9068
:103F00001F9018956F927F928F929F92AF92BF925F
:103F1000CF92DF92EF92FF920F931F93CF93DF9395
:103F2000CDB7DEB762970FB6F894DEBF0FBECDBF38
:103F30008C018091510790915207892B39F0E091C3
:103F40004D07F0914E078081811106C060E070E05E
:103F500087E697E00E94210F87E497E027E08D3401
:103F6000920781F060914D0770914E0761157105C0
:103F700031F040915107509152071ADB03C087E49A
:103F800097E004DBF801A480B580F6E3AF16B10436
:103F900070F4B801CE0101962FDBCE0101960E948C
:103FA0002F130E942713CE01019621DB7EC0C5018D
:103FB00065E370E00E94F631A81AB90A95E3C92EAC
:103FC000D12CE12CF12CEA14FB040CF04BC0A7011E
:103FD000662463944A012FEF821A920A9401B80171
:103FE000CE01019636DB8D819E81892B51F065EEE5
:103FF00074E089819A810E94333477247394892BE9
:1040000009F0712CCE010196F2DA7110612CA40135
:10401000C814D904F9F69601A701B801CE0101969A
:10402000662089F016DBBE016F5F7F4FCE010796D9
:10403000E3DACE0107960E942F130E942713CE01C8
:104040000796D5DA05C005DBCE0101960E9427133D
:10405000CE010196CCDA85E3E80EF11CE5E3CE0E45
:10406000D11CB1CFF80124813581C90165E370E02D
:104070000E94F6310097C9F0A901481B590BB801FD
:10408000CE010196E6DABE016F5F7F4FCE01079643
:10409000B3DACE0107960E942F130E942713CE0198
:1040A0000796A5DACE010196A2DA6DE477E0CE019B
:1040B0000796A2DAAB84BC8400E010E0E12CF12C7E
:1040C0000A151B0524F50F5F1F4FA8014150510928
:1040D0009801BE01695F7F4FCE010196BADA8D81EA
:1040E0009E81892B51F065EE74E089819A810E944E
:1040F0003334DD24D394892B09F0D12CCE010196E1
:1041000076DADD20E9F2FFEFEF1AFF0AD9CFCE0110
:1041100007966DDA8701015011092FE1E216F104CB
:104120000CF440C065EE74E0CE0101967EDAE090BA
:104130005107F0905207E114F10479F1C0904D0756
:10414000D0904E0769817A81C6010E94523400974F
:1041500021F0BC016C197D0902C06FEF7FEF6F5F2A
:104160007F4FD9F0E616F70608F4B701A701461B02
:10417000570B50935207409351076C0D7D1DC6019C
:104180000E944334E0914D07F0914E078091510712
:1041900090915207E80FF91F1082CE01019627DA9D
:1041A0007801B8CF109274071092730783E0EE0C79
:1041B000FF1C8A95E1F7F0927607E09275078FEF82
:1041C0009FEF90937A078093790790937807809375
:1041D000770781E080937B0768018FEFC816D806C8
:1041E00009F47CC06DE477E0CE01079605DAA601FC
:1041F000BE01695F7F4FCE0101964FD2CE01079677
:10420000F6D98091750790917607089710927407F8
:1042100010927307909376078093750767E477E0B1
:10422000CE010796E9D9A601BE01695F7F4FCE0195
:104230000D9633D22D813E8189899A8928173907B5
:1042400019F589819A816D857E85009719F0611530
:104250007105A9F46115710551F02115310539F089
:10426000FB01808190E09195819591090AC00097AA
:1042700069F0232B59F0FC01808190E002C00E947C
:10428000333411E0892B19F010E001C011E0CE01A8
:104290000D96ADD9CE010796AAD9111118C040913B
:1042A000750750917607E12CF12C08E010E020E42E
:1042B00031E060E070E087E697E00E94E80F4D8112
:1042C0005E8169817A8187E697E00E944F18CE016E
:1042D00001968DD9F1E0CF1AD1087FCF62960FB643
:1042E000F894DEBF0FBECDBFDF91CF911F910F912C
:1042F000FF90EF90DF90CF90BF90AF909F908F9006
:104300007F906F900895CF92DF92EF92FF920F937C
:104310001F93CF93DF93CDB7DEB72C970FB6F894EA
:10432000DEBF0FBECDBF6B017C018A0169EB74E07B
:10433000CE0107967AD9B701A601CE010796F6D825
:104340006EED74E0CE0107960E943F1320E030E04E
:1043500040E151E4C701B6010E94283020E030E07E
:1043600040EA50E40E948E3120E030E040E052E428
:104370000E942A31AB01BC01CE010796D7D863EE6B
:1043800074E0CE0107960E943F1367EE74E0CE0101
:1043900007960E943F13B801CE0107960E944D1365
:1043A00069E075E0CE0107960E943F13BE01695F88
:1043B0007F4FCE01019620D9CE010196A3DDCE011B
:1043C000019615D9CE01079612D92C960FB6F894FE
:1043D000DEBF0FBECDBFDF91CF911F910F91FF9038
:1043E000EF90DF90CF900895CF92DF92EF92FF92FF
:1043F0000F931F93CF93DF93CDB7DEB72C970FB6F4
:10440000F894DEBF0FBECDBF6B017C018A016BE06B
:1044100075E0CE01079609D9B701A601CE0107962E
:1044200085D86EED74E0CE0107960E943F1320E020
:1044300030E040E151E4C701B6010E94283020E09D
:1044400030E040EA50E40E948E3120E030E040E06D
:1044500052E40E942A31AB01BC01CE01079666D816
:1044600063EE74E0CE0107960E943F1360E375E0AF
:10447000CE0107960E943F13B801CE0107960E9415
:104480004D1369E075E0CE0107960E943F13BE010F
:10449000695F7F4FCE010196AFD8CE01019632DD24
:1044A000CE010196A4D8CE010796A1D82C960FB6BE
:1044B000F894DEBF0FBECDBFDF91CF911F910F915A
:1044C000FF90EF90DF90CF900895CF92DF92EF9220
:1044D000FF920F931F93CF93DF93CDB7DEB72C9747
:1044E0000FB6F894DEBF0FBECDBF6B017C018A0111
:1044F00062E575E0CE01079698D8B701A601CE0116
:10450000079614D86EED74E0CE0107960E943F1313
:1045100020E030E040E151E4C701B6010E942830BC
:1045200020E030E040EA50E40E948E3120E030E0AC
:1045300040E052E40E942A31AB01BC01CE01079653
:104540000E94961A63EE74E0CE0107960E943F1314
:1045500067E775E0CE0107960E943F13B801CE01D0
:1045600007960E944D1369E075E0CE0107960E9400
:104570003F13BE01695F7F4FCE0101963DD8CE014A
:104580000196C0DCCE01019632D8CE0107962FD815
:104590002C960FB6F894DEBF0FBECDBFDF91CF9142
:1045A0001F910F91FF90EF90DF90CF900895CF92E1
:1045B000DF92EF92FF920F931F93CF93DF93CDB7CC
:1045C000DEB72C970FB6F894DEBF0FBECDBF6B01E0
:1045D0007C018A0169E975E0CE01079626D8B7010A
:1045E000A601CE0107960E94961A6EED74E0CE01E8
:1045F00007960E943F1320E030E040E151E4C701FC
:10460000B6010E94283020E030E040EA50E40E94E9
:104610008E3120E030E040E052E40E942A31AB01CC
:10462000BC01CE0107960E94961A63EE74E0CE019B
:1046300007960E943F136EEB75E0CE0107960E942D
:104640003F13B801CE0107960E944D1369E075E053
:10465000CE0107960E943F13BE01695F7F4FCE01D6
:1046600001960E94FC1ACE0101964CDCCE01019607
:104670000E94F71ACE0107960E94F71A2C960FB6E1
:10468000F894DEBF0FBECDBFDF91CF911F910F9188
:10469000FF90EF90DF90CF9008953F924F925F92FE
:1046A0006F927F928F929F92AF92BF92CF92DF9242
:1046B000EF92FF920F931F93CF93DF9300D000D020
:1046C000CDB7DEB77C016B013A0100E010E0512C60
:1046D000812CA12CB12C302E412EF60184819581A4
:1046E0000817190788F50F5F1F4F9801432D542DA8
:1046F000B601CE0101960E94291B8D819E81892BD6
:1047000051F065EE74E089819A810E9433349924D6
:104710009394892B09F0912CCE0101960E94F71AEF
:104720009920C9F2C5010196A614B70421F0502EB4
:10473000812E5C01D0CF232D342D452D582DB6016F
:10474000C7010E94291B05C069EC72E0C7010E94E5
:10475000151BC70126960FB6F894DEBF0FBECDBF5E
:10476000DF91CF911F910F91FF90EF90DF90CF904D
:10477000BF90AF909F908F907F906F905F904F9081
:104780003F9008953FB7F8948091B8079091B9078A
:10479000A091BA07B091BB0726B5A89B05C02F3FD3
:1047A00019F00196A11DB11D3FBFBA2FA92F982F57
:1047B0008827820F911DA11DB11DBC01CD0142E0D2
:1047C000660F771F881F991F4A95D1F708951F928A
:1047D0000F920FB60F9211242F933F938F939F93B5
:1047E000AF93BF938091E6059091E705A091E8050E
:1047F000B091E9053091B70723E0230F2D3720F45E
:104800000196A11DB11D05C026E8230F0296A11D2A
:10481000B11D2093B7078093E6059093E705A09319
:10482000E805B093E9058091B8079091B907A09188
:10483000BA07B091BB070196A11DB11D8093B807BF
:104840009093B907A093BA07B093BB07BF91AF91FC
:104850009F918F913F912F910F900FBE0F901F90BE
:104860001895CF93DF93CDB7DEB762970FB6F89464
:10487000DEBF0FBECDBF789484B5826084BD84B5A1
:10488000816084BD85B5826085BD85B5816085BD4B
:1048900080916E00816080936E0010928100809103
:1048A000810082608093810080918100816080938B
:1048B0008100809180008160809380008091B100B0
:1048C00084608093B1008091B00081608093B000DB
:1048D000809191008260809391008091910081602D
:1048E00080939100809190008160809390008091EE
:1048F000A10082608093A1008091A10081608093DB
:10490000A1008091A00081608093A000809121018E
:104910008260809321018091210181608093210137
:104920008091200181608093200180917A008460D1
:1049300080937A0080917A00826080937A008091DF
:104940007A00816080937A0080917A0080688093F9
:104950007A001092C100E091AE06F091AF0612E02D
:104960001083E091AA06F091AB061082E091AC06AC
:10497000F091AD068FEC80831092B606E091B206FE
:10498000F091B30686E08083E091B006F091B10625
:10499000808180618083E091B006F091B1068081D2
:1049A00088608083E091B006F091B10680818068D4
:1049B0008083E091B006F091B10680818F7D808385
:1049C0000E94E1170E94E11768EC70E080E090E03F
:1049D0000E94141710938107E0918207F0918307DA
:1049E000908180918E0789238083E0918407F091E4
:1049F0008507908180918F078923808381E082B928
:104A0000E0918607F0918707908180919007892334
:104A10008083E0918607F0918707908180918C07D1
:104A2000892B8083E0918407F091850790818091A4
:104A30008B07892B808312B8E0918607F091870756
:104A400090818091900789238083E0918607F0917F
:104A50008707908180918C07892B808362E370E0C7
:104A600080E090E00E941417E0918407F0918507A0
:104A7000908180918F078923808388E282B9E091B9
:104A80008607F09187079081809190078923808322
:104A9000E0918607F0918707908180918C07892BA0
:104AA0008083E0918407F0918507908180918B0746
:104AB000892B808312B8E0918607F0918707908157
:104AC0008091900789238083E0918607F091870782
:104AD000908180918C07892B8083E0918407F091ED
:104AE0008507908180918F078923808390EC92B90C
:104AF000E0918607F09187072081809190078223BB
:104B00008083E0918607F0918707208180918C0750
:104B1000822B8083E0918407F0918507208180912A
:104B20008B07822B808383E282B9E0918607F09124
:104B3000870720818091900782238083E0918607F8
:104B4000F0918707208180918C07822B8083E091F0
:104B50008407F0918507208180918F0782238083CD
:104B600081EC82B9E0918607F091870720818091DE
:104B7000900782238083E0918607F0918707208148
:104B800080918C07822B8083E0918407F0918507C8
:104B9000208180918B07822B808380E182B9E09114
:104BA0008607F09187072081809190078223808378
:104BB000E0918607F0918707208180918C07822BF6
:104BC0008083E0918407F0918507208180918F0791
:104BD0008223808312B8E0918607F09187072081B5
:104BE0008091900782238083E0918607F091870768
:104BF000208180918C07822B808385EC82B9E091A3
:104C00008607F09187072081809190078223808317
:104C1000E0918607F0918707208180918C07822B95
:104C20008083E0918407F0918507208180918B0734
:104C3000822B80832BE222B9E0918607F0918707CF
:104C400030818091900783238083E0918607F091E3
:104C50008707308180918C07832B808322B9E09174
:104C60008607F091870720818091900782238083B7
:104C7000E0918607F0918707208180918C07822B35
:104C80008083E0918407F0918507208180918F07D0
:104C90008223808387EC82B9E0918607F0918707B1
:104CA00020818091900782238083E0918607F09194
:104CB0008707208180918C07822B8083E091840775
:104CC000F0918507208180918B07822B808392B998
:104CD000E0918607F0918707908180919007892362
:104CE0008083E0918607F0918707908180918C07FF
:104CF000892B8083E0918407F091850790818091D2
:104D00008F078923808386E382B9E0918607F0913B
:104D1000870790818091900789238083E09186079F
:104D2000F0918707908180918C07892B8083E09197
:104D30008407F0918507908180918B07892B808370
:104D400088E882B9E0918607F09187079081809189
:104D5000900789238083E0918607F09187079081EF
:104D600080918C07892B8083E0918407F0918507DF
:104D7000908180918F07892380838AE382B9E091B3
:104D80008607F0918707908180919007892380831F
:104D9000E0918607F0918707908180918C07892B9D
:104DA0008083E0918407F0918507908180918B0743
:104DB000892B808385E582B9E0918607F09187078A
:104DC00090818091900789238083E0918607F091FC
:104DD0008707908180918C07892B8083E0918407DD
:104DE000F0918507908180918F078923808312B885
:104DF000E0918607F0918707908180919007892341
:104E00008083E0918607F0918707908180918C07DD
:104E1000892B808381EB82B9E0918607F091870727
:104E200090818091900789238083E0918607F0919B
:104E30008707908180918C07892B8083E09184077C
:104E4000F0918507908180918B07892B808312B820
:104E5000E0918607F09187079081809190078923E0
:104E60008083E0918607F0918707908180918C077D
:104E7000892B80838BE182B9E0918607F0918707C7
:104E800090818091900789238083E0918607F0913B
:104E90008707908180918C07892B8083E09184071C
:104EA000F0918507908180918F078923808387EB1C
:104EB00082B9E0918607F0918707908180919007F1
:104EC00089238083E0918607F09187079081809104
:104ED0008C07892B8083E0918407F091850790816E
:104EE00080918B07892B808387E082B9E0918607C8
:104EF000F091870790818091900789238083E091CA
:104F00008607F0918707908180918C07892B808399
:104F1000E0918407F0918507908180918F07892324
:104F2000808381E182B9E0918607F09187079081C3
:104F30008091900789238083E0918607F09187070D
:104F4000908180918C07892B8083E0918407F09178
:104F50008507908180918B07892B808312B8E0911F
:104F60008607F0918707908180919007892380833D
:104F7000E0918607F0918707908180918C07892BBB
:104F8000808366E970E080E090E00E941417E09171
:104F90008407F0918507908180918F078923808312
:104FA00089E282B9E0918607F0918707908180912C
:104FB000900789238083E0918607F091870790818D
:104FC00080918C07892B8083E0918407F09185077D
:104FD000908180918B07892B808312B8E09186079E
:104FE000F091870790818091900789238083E091D9
:104FF0008607F0918707908180918C07892B8083A9
:1050000064EF71E080E090E00E9414170FE311E07C
:105010002FEE30E040E050E060E070E087E697E09F
:105020000E94A30761E087E697E00E94DF0D64E934
:1050300072E0CE0101960E94151BCE0101960E94DE
:10504000821FCE0101960E94F71A10E061E0812FC5
:105050000E94D81660E0812F0E94AA161F5F1431AB
:10506000A9F710E261E0812F0E94D81660E0812F3D
:105070000E94AA161F5F1633A9F76AEC72E0CE01F0
:1050800001960E94151BCE0101960E94821FCE013F
:1050900001960E94F71A11E01093E40566E38EEA88
:1050A00097E00E947717811111C060EF72E0CE0186
:1050B00001960E94151BCE0101960E94821FCE010F
:1050C00001960E94F71A1092E30525C062E173E091
:1050D000CE0107960E94151B8EEA97E00E940514E8
:1050E00060E170E0CE0107960E944D13BE01695F3A
:1050F0007F4FCE0101960E94FC1ACE0101960E94BC
:10510000821FCE0101960E94F71A1093E305CE018B
:1051100007960E94F71A67E385EA97E00E947717DF
:10512000811111C06EE373E0CE0101960E94151B40
:10513000CE0101960E94821FCE0101960E94F71AAD
:105140001092E20526C060E673E0CE0107960E9449
:10515000151B85EA97E00E94051460E170E0CE011E
:1051600007960E944D13BE01695F7F4FCE010196E5
:105170000E94FC1ACE0101960E94821FCE01019668
:105180000E94F71A81E08093E205CE0107960E9403
:10519000F71A68E38CE997E00E947717811111C034
:1051A0006CE873E0CE0101960E94151BCE010196BA
:1051B0000E94821FCE0101960E94F71A1092E1050B
:1051C00026C06EEA73E0CE0107960E94151B8CE99B
:1051D00097E00E94051460E170E0CE0107960E94FE
:1051E0004D13BE01695F7F4FCE0101960E94FC1AEC
:1051F000CE0101960E94821FCE0101960E94F71AED
:1052000081E08093E105CE0107960E94F71A69E3D9
:1052100083E997E00E947717811111C06AED73E06E
:10522000CE0101960E94151BCE0101960E94821F9D
:10523000CE0101960E94F71A1092E00526C06CEF8D
:1052400073E0CE0107960E94151B83E997E00E9448
:10525000051460E170E0CE0107960E944D13BE0177
:10526000695F7F4FCE0101960E94FC1ACE01019624
:105270000E94821FCE0101960E94F71A81E080935E
:10528000E005CE0107960E94F71A11E0CC24CA94DB
:1052900083E0D82EE12CF12C8091E505811110924C
:1052A0007A008EE996E00E94AA18181619060CF0EA
:1052B00052C069EC72E0CE0101960E94151B0E945B
:1052C000291497FD0CC08F83188641E050E0BE0181
:1052D000695F7F4FCE0101960E94691AF0CF68E2A4
:1052E00074E0CE0107960E94151B4D815E81698195
:1052F0007A81CE0107960E94691A811104C0CE01FD
:1053000007960E94C61ABE01695F7F4FCE010D96B7
:105310000E94FC1ACE0107960E94F71ACE01019650
:105320000E94F71A29893A892150310940E050E05A
:10533000BE01635F7F4FCE0101960E94291BCE0103
:1053400001960E94821FCE0101960E94F71ACE019B
:105350000D960E94F71A8091E3058823C9F18EEA21
:1053600097E00E94D8134B015C018EEA97E00E94FF
:105370004E179C01A4E6B0E05DD7A70196011CD7AB
:1053800029013A01213737410CF120E030E040E8B3
:105390005FE3C501B401F7D587FF18C066E38EEA65
:1053A00097E00E94771781112AC01092E30560EF01
:1053B00072E0CE0101960E94151BCE0101960E945B
:1053C000821FCE0101960E94F71A2EC0A20129C0A9
:1053D00066E38EEA97E00E947717882329F11093FD
:1053E000E30561E374E0CE0101960E94151BCE0136
:1053F00001960E94821FCE0101960E94F71A8EEA42
:1054000097E00E94D8134B015C018EEA97E00E945E
:105410004E179C01A4E6B0E00DD7A7019601CCD6AB
:10542000A901C501B401C3D88091E205882309F41C
:105430004FC085EA97E00E94D8134B015C0185EAD2
:1054400097E00E944E179C01A4E6B0E0F3D6A701B6
:105450009601B2D629013A0121373741BCF120E04B
:1054600030E040E85FE3C501B4018DD587FF2EC071
:1054700067E385EA97E00E947717811111C01092C7
:10548000E2056EE373E0CE0101960E94151BCE018A
:1054900001960E94821FCE0101960E94F71A45C014
:1054A00085EA97E00E94D8134B015C0185EA97E0FA
:1054B0000E944E179C01A4E6B0E0BCD6A70196015D
:1054C0007BD6A901C501B40172D82FC0A20129C0A1
:1054D00067E385EA97E00E947717882331F11093FC
:1054E000E20563E574E0CE0101960E94151BCE0132
:1054F00001960E94821FCE0101960E94F71A85EA4A
:1055000097E00E94D8134B015C0185EA97E00E9466
:105510004E179C01A4E6B0E08DD6A70196014CD6AB
:10552000A901C501B4010E9465228091E10588238B
:10553000C9F18CE997E00E94D8134B015C018CE91A
:1055400097E00E944E179C01A4E6B0E073D6A70135
:10555000960132D629013A01213737410CF120E07A
:1055600030E040E85FE3C501B4010DD587FF18C006
:1055700068E38EEA97E00E94771781112AC01092A3
:10558000E1056CE873E0CE0101960E94151BCE0187
:1055900001960E94821FCE0101960E94F71A2FC029
:1055A000A20129C068E38CE997E00E94771788235D
:1055B00031F11093E10565E774E0CE0101960E9498
:1055C000151BCE0101960E94821FCE0101960E94FA
:1055D000F71A8CE997E00E94D8134B015C018CE923
:1055E00097E00E944E179C01A4E6B0E023D6A701E5
:1055F0009601E2D5A901C501B4010E94F421809170
:10560000E0058823C9F183E997E00E94D8134B0194
:105610005C0183E997E00E944E179C01A4E6B0E08C
:1056200009D6A7019601C8D529013A01213737418A
:105630000CF120E030E040E85FE3C501B401A3D401
:1056400087FF18C069E38EEA97E00E9477178111FF
:105650002AC01092E0056AED73E0CE0101960E9427
:10566000151BCE0101960E94821FCE0101960E9459
:10567000F71A2FC0A20129C069E38EEA97E00E94C1
:105680007717882331F11093E00567E974E0CE01C4
:1056900001960E94151BCE0101960E94821FCE0129
:1056A00001960E94F71A83E997E00E94D8134B01F4
:1056B0005C0183E997E00E944E179C01A4E6B0E0EC
:1056C000B9D5A701960178D5A901C501B4010E94F9
:1056D000832160ED77E080E090E00E9414170E9443
:1056E0004E19DACD87E497E00E94F71A8DE497E02F
:1056F0000C94F71ABF92CF92DF92EF92FF920F9322
:105700001F93CF93DF93EEE9F6E01382128288EEC7
:1057100093E0A0E0B0E084839583A683B78320E282
:1057200032E03183208325EC30E03587248724EC78
:1057300030E03787268720EC30E0318B208B21EC5E
:1057400030E0338B228B22EC30E0358B248B26EC3F
:1057500030E0378B268B118E128E138E148EEBE376
:10576000F7E01382128284839583A683B78382E352
:1057700092E091838083AEEAB7E013961C921E926A
:1057800012978CE792E011969C938E931696FC9359
:10579000EE931597A5EAB7E013961C921E92129706
:1057A00011969C938E931696FC93EE931597ACE905
:1057B000B7E013961C921E92129711969C938E93AB
:1057C0001696FC93EE931597A3E9B7E013961C92F7
:1057D0001E92129711969C938E931696FC93EE93BD
:1057E0001597C7E6D7E01B821A8280EFE82EF12CCE
:1057F000FD82EC8200E411E01F830E83F986E886C7
:105800001B870A871D8A1D861C861F861E86BB2451
:10581000B394BC8ACC24CA94DC2CDB8ACA8AD98A89
:10582000C88ABE8A1F8A198E188E84E492E09983F2
:10583000888386E38BA7E5E1F8E0E491F0E0EE0FE2
:10584000FF1FEE53F84FA591B491BC8FAB8FE4E1ED
:10585000F8E0E491F0E0EE0FFF1FEE53F84F859172
:1058600094919E8F8D8FE3E1F8E0E491F0E0EE0FEC
:10587000FF1FEE53F84F8591949198A38F8FE2E12B
:10588000F8E0E491F0E0EE0FFF1FEE53F84F859142
:1058900094919AA389A3E5EBF7E034913BA3E4EB61
:1058A000F7E024912CA3E3EBF7E094919DA3E2EBC6
:1058B000F7E084918EA3432F40954FA3E22FE0950C
:1058C000E8A7E92FE095E9A7E82FE095EAA7EC9192
:1058D000E32BEC93ED8DFE8D90818CA1892B808341
:1058E000EF8DF8A190818DA1892B8083E9A1FAA188
:1058F00090818EA1892B808361E089E30E94D81674
:1059000061E088E30E94D81661E087E30E94D81620
:1059100061E086E30E94D81661E086E30E94AA1641
:1059200061E086E30E94D8168FEF81B91D8A1D863B
:105930001C861F861E86BC8AD98AC88AF986E88694
:105940001B870A87A3E5B7E08AE312968C93129728
:105950008BE314968C9314978EE113968C93139784
:105960008FE115968C9315978DE491E017969C9393
:105970008E931697EBEFF7E0E491F0E0EE0FFF1F48
:10598000EE53F84F8591949119969C938E931897A6
:10599000E6E1F8E0E491F0E0EE0FFF1FEE53F84F80
:1059A000859194911B969C938E931A97E7E1F8E06A
:1059B000E491F0E0EE0FFF1FEE53F84F85919491C4
:1059C0001D969C938E931C97EAEFF7E0E491F0E02C
:1059D000EE0FFF1FEE53F84F859194911F969C9305
:1059E0008E931E97EBE9F7E0E4915096EC93509775
:1059F000E6EBF7E0E4915296EC935297E7EBF7E091
:105A0000E4915196EC935197EAE9F7E0E4915396CB
:105A1000EC9353978AE090E08D939C9369EC72E04D
:105A20008DE497E00E94151B69EC72E087E497E033
:105A3000DF91CF911F910F91FF90EF90DF90CF906A
:105A4000BF900C94151BEF920F931F93CF93DF938E
:105A5000E80147FD02C034E001C034E1042E000C2F
:105A6000550B57FF03C0519541955109E32E022F65
:105A7000242FAE012AD0CE01DF91CF911F910F913B
:105A8000EF900895BB274A3031F4992322F4BDE208
:105A9000909581959F4F01C0BB27FB015527AA27F1
:105AA000880F991FAA1FA41710F0A41B83955051AB
:105AB000B9F7A05DAA3308F0A95DA193009779F723
:105AC000B111B1931192CB014EC28F929F92AF92BE
:105AD000BF92CF92DF92EF92FF920F931F93CF93DB
:105AE000DF93CDB7DEB729970FB6F894DEBF0FBEB0
:105AF000CDBF6A01122FB02E2BE3201720F0FF2418
:105B0000F394F00E02C02CE3F22E0F2D27E0AE012D
:105B10004F5F5F4F50D1BC014981842F8970813024
:105B200031F0E1FC06C0E0FE06C090E205C09DE257
:105B300003C09BE201C090E05E2D507143FF3CC06A
:105B4000911102C083E001C084E0811718F4212F75
:105B5000281B01C020E051110BC0F601822F30E25A
:105B6000882319F031938150FBCFC20ED11C20E065
:105B7000992329F0D6019C93F60131966F01C60155
:105B80000396E2FE0AC03EE4D6013C9341E411963E
:105B90004C93119712963C9306C03EE6F601308373
:105BA00041E641833283FC01322F40E2332309F482
:105BB00042C041933150FACF42FF44C0911102C01C
:105BC00083E001C084E0811718F4212F281B01C055
:105BD00020E051110BC0F601822F30E2882319F02A
:105BE00031938150FBCFC20ED11C20E0992329F0C4
:105BF000D6019C93F60131966F01C6010396E2FE31
:105C00000BC039E4D6013C933EE411963C931197C6
:105C100036E412963C9307C039E6F60130833EE63F
:105C2000318336E63283FC01322F40E2332319F010
:105C300041933150FBCFFC01E20FF11D10828EEF3A
:105C40009FEFA6C021E030E0911102C020E030E0DB
:105C5000161617061CF4FB01319602C0E1E0F0E0D5
:105C60002E0F3F1FBB2021F0EB2DF0E0319602C03C
:105C7000E0E0F0E02E0F3F1FE12FF0E02E173F078E
:105C80001CF4121B212F01C020E08E2D887159F4C5
:105C9000F601822F30E2882319F031938150FBCF37
:105CA000C20ED11C20E0992329F0D6019C93F60165
:105CB00031966F0151110BC0F601822F90E38823BA
:105CC00019F091938150FBCFC20ED11C20E00F2D13
:105CD000060F9A81342F307144FF03C0913309F4C9
:105CE0000150101624F4093018F008E001C001E05A
:105CF000AB0177FF02C040E050E0FB01E41BF50B75
:105D0000A1E0B0E0AC0FBD1FEA0FFB1F8EE2A82E92
:105D10004B01801A91080B2D10E011950195110986
:105D20004F3FBFEF5B0721F4D601AC9211966D0196
:105D3000641775072CF08416950614F4818101C050
:105D400080E3415051093196D60111967D014017EB
:105D5000510724F0D6018C936701E2CF64177507D1
:105D600039F4963320F4953319F4311101C081E3ED
:105D7000F6018083F701822F90E2882319F0919336
:105D80008150FBCFF701E20FF11D108280E090E01F
:105D900029960FB6F894DEBF0FBECDBFDF91CF912D
:105DA0001F910F91FF90EF90DF90CF90BF90AF9039
:105DB0009F908F900895283008F027E03327DA016C
:105DC000990F311D87FD916000966105710539F4C9
:105DD00032602E5F3D9330E32A95E1F708959F3FAF
:105DE00030F080387105610509F03C5F3C5F3D9300
:105DF000913008F08068911DDF93CF931F930F932C
:105E0000FF92EF92192F987F9695E92F9695969588
:105E1000E90FFF27EE59FE4F99273327EE24FF2481
:105E2000A701E70105900894079428F4360FE71EB0
:105E3000F81E491F511D660F771F881F991F069472
:105E4000A1F70590079428F4E70EF81E491F561F86
:105E5000C11D770F881F991F661F0694A1F7059033
:105E6000079428F4F80E491F561FC71FD11D880F2D
:105E7000991F661F771F0694A1F70590079420F4D9
:105E8000490F561FC71FD81F990F661F771F881FFE
:105E90000694A9F784911095177041F0D695C7958F
:105EA00057954795F794E7941A95C1F7E8E0F1E024
:105EB00068941590159135916591959105907FE2C3
:105EC0007395E118F10A430B560BC90BD009C0F7C3
:105ED000E10CF11E431F561FC91FD01D7EF4703305
:105EE00011F48A95E6CFE894015030F0080F0AF4D7
:105EF0000027021708F4202F2395022F7A3328F069
:105F000079E37D932A95E9F710C07D932A9589F668
:105F1000069497956795379517951794E118F10AA8
:105F2000430B560BC90BD00998F023957E917395BE
:105F30007A3308F070E37C932013B8F77E91706198
:105F40007D9330F0839571E37D9370E32A95E1F7BB
:105F50001124EF90FF900F911F91CF91DF9199271E
:105F600087FD90950895DC01FC01672F71917723DF
:105F7000E1F7329704C07C916D9370836291AE1704
:105F8000BF07C8F3089540D008F481E00895E8946D
:105F900009C097FB3EF490958095709561957F4F71
:105FA0008F4F9F4F9923A9F0F92F96E9BB2793951F
:105FB000F695879577956795B795F111F8CFFAF42F
:105FC000BB0F11F460FF1BC06F5F7F4F8F4F9F4F60
:105FD00016C0882311F096E911C0772321F09EE8BE
:105FE000872F762F05C0662371F096E8862F70E024
:105FF00060E02AF09A95660F771F881FDAF7880FFE
:106000009695879597F90895990F0008550FAA0B53
:10601000E0E8FEEF16161706E807F907C0F01216BB
:106020001306E407F50798F0621B730B840B950BBE
:1060300039F40A2661F0232B242B252B21F4089513
:106040000A2609F4A140A6958FEF811D811D0895B0
:106050000BD078C069D028F06ED018F0952309F0E5
:106060005AC05FC01124A2C07ED0A0F3959FD1F387
:10607000950F50E0551F629FF001729FBB27F00DF6
:10608000B11D639FAA27F00DB11DAA1F649F66274B
:10609000B00DA11D661F829F2227B00DA11D621F9A
:1060A000739FB00DA11D621F839FA00D611D221F54
:1060B000749F3327A00D611D231F849F600D211D38
:1060C000822F762F6A2F11249F5750408AF0E1F0DB
:1060D00088234AF0EE0FFF1FBB1F661F771F881F24
:1060E00091505040A9F79E3F510570F014C05EC01A
:1060F0005F3FECF3983EDCF3869577956795B7950F
:10610000F795E7959F5FC1F7FE2B880F911D969538
:10611000879597F9089597F99F6780E870E060E0A8
:1061200008959FEF80EC089500240A941616170630
:1061300018060906089500240A9412161306140678
:1061400005060895092E0394000C11F4882352F0DB
:10615000BB0F40F4BF2B11F460FF04C06F5F7F4F93
:106160008F4F9F4F089557FD9058440F551F59F07A
:106170005F3F71F04795880F97FB991F61F09F3F34
:1061800079F087950895121613061406551FF2CF5D
:106190004695F1DF08C0161617061806991FF1CFAD
:1061A00086957105610508940895E894BB276627D4
:1061B0007727CB0197F90895052E97FB16F40094E5
:1061C0000FD057FD05D014D007FC02D046F408C00C
:1061D00050954095309521953F4F4F4F5F4F089513
:1061E00090958095709561957F4F8F4F9F4F089543
:1061F000A1E21A2EAA1BBB1BFD010DC0AA1FBB1FCB
:10620000EE1FFF1FA217B307E407F50720F0A21B3C
:10621000B30BE40BF50B661F771F881F991F1A94A9
:1062200069F760957095809590959B01AC01BD01D3
:10623000CF010895A29FB001B39FC001A39F700D2D
:10624000811D1124911DB29F700D811D1124911D7E
:1062500008955058BB27AA270ED074CF65DF30F0C1
:106260006ADF20F031F49F3F11F41EF45ACF0EF490
:10627000E095E7FB50CFE92F76DF80F3BA1762078E
:1062800073078407950718F071F49EF58ECF0EF40E
:10629000E0950B2EBA2FA02D0B01B90190010C0136
:1062A000CA01A0011124FF27591B99F0593F50F44E
:1062B000503E68F11A16F040A22F232F342F4427A6
:1062C000585FF3CF469537952795A795F04053959E
:1062D000C9F77EF41F16BA0B620B730B840BBAF06E
:1062E0009150A1F0FF0FBB1F661F771F881FC2F7D9
:1062F0000EC0BA0F621F731F841F48F487957795ED
:106300006795B795F7959E3F08F0B3CF9395880FA3
:1063100008F09927EE0F9795879508950CD012CF26
:106320000ADF40F001DF30F021F45F3F19F0F3CED7
:1063300051113CCFF6CE17DF98F39923C9F35523BB
:10634000B1F3951B550BBB27AA2762177307840768
:1063500038F09F5F5F4F220F331F441FAA1FA9F31E
:1063600033D00E2E3AF0E0E830D091505040E69510
:10637000001CCAF729D0FE2F27D0660F771F881F71
:10638000BB1F261737074807AB07B0E809F0BB0B60
:10639000802DBF01FF2793585F4F2AF09E3F510584
:1063A00068F0B9CE03CF5F3FECF3983EDCF38695FF
:1063B00077956795B795F7959F5FC9F7880F911DFA
:1063C0009695879597F90895E1E0660F771F881FE6
:1063D000BB1F621773078407BA0720F0621B730B99
:1063E000840BBA0BEE1F88F7E0950895AA1BBB1B20
:1063F00051E107C0AA1FBB1FA617B70710F0A61BC5
:10640000B70B881F991F5A95A9F780959095BC01E5
:10641000CD010895EE0FFF1F881F8BBF0790F691E7
:10642000E02D1994692796276927782787277827E9
:10643000089500DF332312F48A1B9B0B01C0FADEA0
:10644000B7FF0895821B930B08950F931F93CF936B
:10645000DF938230910510F482E090E0E091BE0776
:10646000F091BF0720E030E0A0E0B0E0309719F1F4
:10647000408151810281138148175907C8F0841760
:10648000950769F4109731F012960C9312971396B2
:106490001C9327C00093BE071093BF0722C021158D
:1064A000310519F04217530718F49A01BD01EF01A5
:1064B000DF01F801DBCF21153105F9F0281B390B7D
:1064C0002430310580F48A819B816115710521F0AA
:1064D000FB019383828304C09093BF078093BE0720
:1064E000FE01329644C0FE01E20FF31F81939193A7
:1064F00022503109398328833AC02091BC0730915A
:10650000BD07232B41F42091020230910302309306
:10651000BD072093BC072091000230910102211594
:10652000310541F42DB73EB7409104025091050268
:10653000241B350BE091BC07F091BD07E217F30770
:10654000A0F42E1B3F0B2817390778F0AC014E5FE3
:106550005F4F2417350748F04E0F5F1F5093BD075C
:106560004093BC078193919302C0E0E0F0E0CF013B
:10657000DF91CF911F910F910895CF93DF930097F3
:1065800009F481C0FC01329713821282A091BE07E8
:10659000B091BF07109781F420813181820F931F42
:1065A0002091BC073091BD072817390751F5F093AA
:1065B000BD07E093BC0767C0ED0120E030E0CE17D7
:1065C000DF0740F44A815B819E0141155105F1F0DE
:1065D000EA01F5CFD383C28340815181840F951F97
:1065E000C817D90759F488819981840F951F02969D
:1065F000918380838A819B819383828321153105D6
:1066000029F4F093BF07E093BE073DC0E901FB8387
:10661000EA8349915991C40FD51FEC17FD0761F426
:1066200080819181840F951F0296E9019983888367
:10663000828193819B838A83E0E0F0E012968D91C2
:106640009C911397009719F0FD01DC01F7CF8D9114
:106650009C9111979D012E5F3F4F820F931F2091B8
:10666000BC073091BD072817390769F4309729F422
:106670001092BF071092BE0702C013821282B0931D
:10668000BD07A093BC07DF91CF9108956F927F92D1
:106690008F929F92AF92BF92CF92DF92EF92FF9232
:1066A0000F931F93CF93DF93009781F4CB01DF917A
:1066B000CF911F910F91FF90EF90DF90CF90BF90FF
:1066C000AF909F908F907F906F90BFCEFC01E60FB0
:1066D000F71F9C0122503109E217F30708F4A5C007
:1066E000EC01D9010D911C91119706171707A8F01D
:1066F0000530110508F497C0C8010497861797075D
:1067000008F491C002501109061B170B0193119355
:106710006D937C93CF0131DF86C05B01A01AB10A73
:106720004C01800E911EA091BE07B091BF07612C55
:10673000712CE12CF12C109709F446C08D919C919D
:106740001197A815B905B1F56C0142E0C40ED11C32
:10675000CA14DB0478F14C018A189B08640142E0FA
:10676000C40ED11C1296BC9012971396AC91B5E052
:10677000CB16D10440F0B282A38391828082D901EA
:106780006D937C9309C00E5F1F4F800F911FF9011D
:1067900091838083EB2DFA2FE114F10431F0D701BE
:1067A0001396FC93EE9312973EC0F093BF07E093CD
:1067B000BE0739C06816790608F43C017D011296BF
:1067C0000D90BC91A02DB7CF8091BC079091BD07D3
:1067D00088169906E1F466167706C8F480910002DF
:1067E00090910102009741F48DB79EB74091040249
:1067F00050910502841B950BE817F907B0F4F0934C
:10680000BD07E093BC07F901718360830CC0CB0125
:106810001CDE7C01009749F0A801BE011BD0CE010F
:10682000ACDEC70104C0CE0102C080E090E0DF9181
:10683000CF911F910F91FF90EF90DF90CF90BF907D
:10684000AF909F908F907F906F90089581E090E03F
:10685000F89442C0FB01DC0102C001900D9241504E
:106860005040D8F70895FB01DC018D91019080190B
:106870000110D9F3990B0895FB01DC0101900D92F1
:106880000020E1F70895FB01DC014150504048F041
:1068900001900D920020C9F701C01D924150504057
:1068A000E0F70895FB0151915523A9F0BF01DC01E8
:1068B0004D9145174111E1F759F4CD0101900020A8
:1068C00049F04D9140154111C9F3FB014111EFCF42
:1068D00081E090E00197089514E0C2E1D4E000E087
:1068E00005C0802FFE0196DD2196011DC331D10721
:0A68F00080E00807B1F7F894FFCF2D
:1068FA000000C007800000003F013F01EFEF006089
:10690A00C0A02810001018100001020300000000A7
:10691A00E1184F1879182D19AA1888189C18000020
:10692A000000121AE619681FBA19DE19CA19BB192A
:10693A000000000017064F18681F671FDA0BBA1904
:10694A00AF1EFB05A31E0B06B61EBA19DF0D4504C2
:10695A007110E10AE80F210FBA045B04000000007D
:10696A00401A4F18681F671F00000000841D4F1847
:10697A00681F671F640B9C0B420B4D1D39003800C2
:10698A00370036005B20204F4B20205D20456E618A
:10699A00626C696E6720706F776572736176696E73
:1069AA00672066656174757265732E2E2E2020200D
:1069BA00202020202020202020005B20204F4B2058
:1069CA00205D20456E61626C6564204C6576656C5D
:1069DA00203120706F776572736176696E672E0059
:1069EA005B20494E464F205D20536F696C207365CA
:1069FA006E736F72203120756E706C75676765648F
:106A0A002E005B20204F4B20205D20536F696C20A5
:106A1A0073656E736F72203120636F6E6E65637477
:106A2A0065642E2056657273696F6E3A20005B208A
:106A3A00494E464F205D20536F696C2073656E7313
:106A4A006F72203220756E706C75676765642E00F0
:106A5A005B20204F4B20205D20536F696C207365AB
:106A6A006E736F72203220636F6E6E656374656435
:106A7A002E2056657273696F6E3A20005B20494E6C
:106A8A00464F205D20536F696C2073656E736F7279
:106A9A00203320756E706C75676765642E005B2005
:106AAA00204F4B20205D20536F696C2073656E73F5
:106ABA006F72203320636F6E6E65637465642E2077
:106ACA0056657273696F6E3A20005B20494E464FD5
:106ADA00205D20536F696C2073656E736F7220346A
:106AEA0020756E706C75676765642E005B20204F99
:106AFA004B20205D20536F696C2073656E736F7233
:106B0A00203420636F6E6E65637465642E2056654B
:106B1A007273696F6E3A200053657269616C3A202C
:106B2A00005B20494E464F205D20536F696C2073ED
:106B3A00656E736F72203120636F6E6E6563746564
:106B4A00642E005B20494E464F205D20536F696CCE
:106B5A002073656E736F72203220636F6E6E656389
:106B6A007465642E005B20494E464F205D20536FAA
:106B7A00696C2073656E736F72203320636F6E6E5B
:106B8A0065637465642E005B20494E464F205D2084
:106B9A00536F696C2073656E736F72203420636F54
:106BAA006E6E65637465642E005B20204F4B202057
:106BBA005D20536F696C2073656E736F7220342089
:106BCA0074656D70657261747572653A2000204350
:106BDA002C200020467C005B20204F4B20205D208B
:106BEA00536F696C2073656E736F722034206D6FFA
:106BFA006973747572653A200025005B20204F4B3B
:106C0A0020205D20536F696C2073656E736F72204C
:106C1A00332074656D70657261747572653A20000F
:106C2A005B20204F4B20205D20536F696C207365D9
:106C3A006E736F722033206D6F6973747572653A63
:106C4A0020005B20204F4B20205D20536F696C2071
:106C5A0073656E736F7220322074656D7065726130
:106C6A00747572653A20005B20204F4B20205D200E
:106C7A00536F696C2073656E736F722032206D6F6B
:106C8A006973747572653A20005B20204F4B20208F
:106C9A005D20536F696C2073656E736F72203120AB
:106CAA0074656D70657261747572653A20005B2057
:106CBA00204F4B20205D20536F696C2073656E73E3
:106CCA006F722031206D6F6973747572653A200096
:00000001FF
